:020000040800F2
:100000003011002001010008FB370008C528000856
:10001000F9370008350F0008A1640008000000004F
:10002000000000000000000000000000CD490008B2
:10003000931A000800000000653D0008CD4C000840
:100040001B010008593B00081B0100081B010008A8
:100050001B0100081B0100081B0100081B01000810
:100060001B0100081B0100081B0100081B01000800
:100070001B0100081B0100084D1500081B010008AA
:100080001B0100081B0100083D0700081B010008B8
:100090001B0100081B0100081B0100081B010008D0
:1000A0003D4D0008294E00081B0100081B010008F7
:1000B0002D4E00081D510008795300081B0100084F
:1000C0001B0100081B0100081B0100081B010008A0
:1000D0001B010008995F00081B0100081B010008B4
:1000E0001B0100081B0100081B010008DFF80CD0F1
:1000F00000F0E6FA00480047AD7500083011002016
:100100000648804706480047FEE7FEE7FEE7FEE7B1
:10011000FEE7FEE7FEE7FEE7FEE7FEE7ED4C000840
:10012000ED0000082DE9F0410024061B254671F181
:10013000000605DA01240027D0EB070067EB010178
:10014000161E73F1000605DA0027D2EB070201251F
:1001500067EB030300F0D0F986460E4617469C462F
:10016000AC4204D00025D0EB050E65EB010624B1AE
:100170000020D2EB000760EB030C704631463A4694
:100180006346BDE8F08140EA01039B0703D009E024
:1001900008C9121F08C0042AFAD203E011F8013B73
:1001A00000F8013B521EF9D2704780EA010210B5F7
:1001B00002F00043400022D04A001FD0010E01EBA4
:1001C0001261C0F35600C2F3560240F4000042F43C
:1001D0000002A0FB022000047F39140400D0401C60
:1001E00050EA124001D44000491EC2B20C0604EB92
:1001F000D010401C4008802A02D003E0002010BD2F
:1002000020F00100002900DA0020184310BD2DE97C
:10021000FE4F81EA030404F0004421F00041009401
:100220004FF0000B23F0004350EA01045ED052EA85
:1002300003045BD0C3F30A54C1F30A552C44A4F25F
:10024000F3340194A0FB0254C1F3130141F4801173
:10025000C3F3130343F4801301FB024400FB034E7A
:10026000840A970A44EA815447EA8357A4FB076843
:1002700002958D0A05FB07854FEA932C04FB0C546D
:100280002705029D4FEA065847EA1637B5EB0805E1
:100290006EEB070C870E920E47EA811742EA831233
:1002A000A7FB0201B6EB0B0164EB00042B0D43EA44
:1002B0000C335E1844EB1C50DA465146E7FB020152
:1002C000C5F313044FEA0B3343EA14534FEA0432E5
:1002D000019C43EA0603A4F10C040294009CCDE9BE
:1002E00000B400F09FF903B0BDE8F08F0020014694
:1002F000F9E72DE9F04D81EA030404F0004B21F009
:10030000004514464FF0000A23F0004150EA050270
:1003100020D054EA01021DD0C5F30A570246C5F3A6
:100320001303C1F31300C1F30A5640F4801543F4DC
:100330008013A7EB0608101BD64608F2FD3873EBB6
:10034000050002D308F1010801E092185B41B8F101
:10035000000F03DA00200146BDE8F08D00204FF4C5
:100360008011064684460EE0171B73EB050705D384
:10037000121B63EB050306434CEA010C49084FEAE4
:10038000300092185B4150EA0107EDD152EA0300B8
:1003900012D082EA040083EA0501084305D0101B4D
:1003A000AB4106D20122002306E000224FF00043B9
:1003B00002E06FF0010253101AEB06004CEB0851FB
:1003C00010EB0A0041EB0B01BDE8F04D00F01BB94A
:1003D00070B521F0004303430CD0C1F30A5500244B
:1003E000D5EB040564EB0403D617AD1AB34102DB69
:1003F0000020014670BD201841EB025170BDC10FB5
:1004000080EAE0700844CA079623002100F0CDB8C6
:1004100096230022114600F0C8B80EB5C10F80EA3D
:10042000E0700844CA07002140F233438DE80E0013
:100430000A460B4600F0F6F803B000BD0EB540F2D8
:10044000334102910021CDE900110A460B4600F02C
:10045000E9F803B000BD00F0004220F00040C10DFB
:10046000C0F3160040F400007F2901DA0020704735
:10047000962903DCC1F19601C84001E09639884015
:10048000002AF4D04042704770B5C1F30A5201F01F
:1004900000450024C1F3130140F2FF3341F4801101
:1004A0009A4201DA002070BD40F233439A42A2F230
:1004B000334203DC524200F05FF800E090402C43EE
:1004C000F1D0404270BDC1F30A5210B5C1F313011F
:1004D00040F2FF3341F480119A4201DA002010BD4E
:1004E00040F233439A42A2F2334203DC524200F01C
:1004F00043F810BD904010BD2DE9F05F0546002087
:1005000092469B4688460646814640241BE0284684
:1005100041464746224600F02FF853465A46C01A35
:10052000914110D311461846224600F016F82D1AB4
:1005300067EB01084F4622460120002100F00DF82C
:1005400017EB00094E41201EA4F10104DFDC4846F0
:1005500031462A464346BDE8F09F202A04DB203A74
:1005600000FA02F1002070479140C2F1200320FA06
:1005700003F3194390407047202A04DB203A21FA04
:1005800002F00021704721FA02F3D040C2F12002AC
:1005900091400843194670470029A8BF7047401C86
:1005A000490008BF20F00100704710B4B0FA80FC89
:1005B00000FA0CF050EA010404BF10BC704749B1C6
:1005C000CCF1200421FA04F411FA0CF118BF012136
:1005D00021430843A3EB0C01CB1D4FEA00614FEA16
:1005E000102042BF002010BC704700EBC3501044E5
:1005F0000029A4BF10BC7047401C490008BF20F070
:10060000010010BC704710B5141E73F1000408DA25
:10061000401C41F1000192185B411A4301D120F0C6
:10062000010010BD2DE9F04D92469B4611B1B1FA83
:1006300081F202E0B0FA80F220329046FFF78DFF9F
:1006400004460F4640EA0A0041EA0B0153465A4667
:10065000084313D0114653EA010019D0C8F14002F3
:100660005046FFF789FF05460E465046594642461A
:10067000FFF773FF084305D0012004E02046394608
:10068000BDE8F08D0020054346EAE0762C43374371
:100690000A986305E40AA0EB08000022FD0A44EA78
:1006A00047540A3002D500200146E9E70105101938
:1006B0006941DDE9084500196941BDE8F04DA2E74F
:1006C000064C074D06E0E06840F0010394E807009F
:1006D00098471034AC42F6D3FFF70CFD7C99000824
:1006E0009C99000870B58C1810F8015B15F0070391
:1006F00001D110F8013B2A1106D110F8012B03E0BB
:1007000010F8016B01F8016B5B1EF9D12B0705D4C2
:100710000023521E0DD401F8013BFAE710F8013B0B
:10072000CB1A921C03E013F8015B01F8015B521E27
:10073000F9D5A142D8D3002070BD000070B54C4C53
:100740004FF490652946204600F015FA002864D041
:100750002946204600F0A2F846490888401C088037
:100760000121204600F0E6FA434942F21072B1F846
:100770005000904202D2401CA1F8500007F0FEF851
:100780003E4DB5F91410B5F9120005F0BBFF3C4C15
:10079000A5F856002080A16820468847A088A5F8C3
:1007A000580003F093F807F0E5F9364E364C3078F0
:1007B000082833D045F6AC30606042F6EF60A060A8
:1007C00042F2C400E0603148008A2080208E6080C0
:1007D000A16B2D488847208E69882D4C08444FF620
:1007E000FF7101EA80006887207A4FF0000540071A
:1007F0001DD501F0DDFA274949F6A24008802648B8
:1008000040F21A62C188491C89B2C180914204D366
:10081000A16821F00401A160C58070BD41F2130000
:1008200060604FF48060A06040F61B50CAE73078EB
:100830000A2818D2DFE800F0170613050A050D177D
:100840001113EAE7BDE8704006F006B908F078F940
:1008500005E0BDE8704002F083BD06F083FCBDE812
:10086000704007F0DFBA00F0FDFB84F8B65070BDB1
:1008700000240140280700204801002064000020D7
:10088000480700201F070020E4000020F801002096
:10089000A8020020442C0140680900206FEA1121C1
:1008A000016070470029816802D041F0010101E038
:1008B00021F00101816070470029816802D041F474
:1008C000807101E021F48071816070472DE9F04171
:1008D000824E92B0304600F00BF90BA800F039FAC6
:1008E00001214FF4C06003F0D1FA00248DF83140AB
:1008F0004FF46020CDE90D044FF4A0204FF009081B
:100900000B9001278DF83C808DF830700BA9304694
:1009100000F080F9724D8DF831408DF830708DF80F
:100920003C700BA9284600F075F901231A460F21E7
:10093000304600F0C0F9022201231146304600F093
:10094000BAF9012303220021304600F0B4F9012353
:1009500004221946304600F0AEF9012305220B218E
:10096000304600F0A8F9012306220421304600F0A9
:10097000A2F9012307220821304600F09CF9012347
:1009800008220321304600F096F9012309220A21AA
:10099000304600F090F90121304600F084F9012141
:1009A000284600F080F901231A460521304600F060
:1009B00055F901231A460621284600F04FF9002177
:1009C000304600F0CBF84FF4E041284600F0C6F87E
:1009D0000121304600F0B8F80121284600F0B4F8B3
:1009E0000121304600F0A6F80121284600F0A2F8C7
:1009F0000121304600F09EF90121284600F09AF9C5
:100A000040F61451374804F08EFF12208DF8400054
:100A100002208DF841008DF842408DF8437010A8F7
:100A200002F018FF01224FF49061304600F0E8F820
:100A300001213046FFF740FF01213046FFF732FF2A
:100A400001212846FFF72EFF304600F06EF93046B0
:100A500000F09FF80028FAD1304600F075F93046D2
:100A600000F082F80028FAD1284600F05EF9284606
:100A700000F08FF80028FAD1284600F065F92846E2
:100A800000F072F80028FAD10121084603F0DAF9E3
:100A9000154D284600F096FD684600F03EFE0F48D2
:100AA00001A94C300090114881E811018020CDE966
:100AB00004404000069080000790202008904FF4EA
:100AC0004050CDE909046946284600F009FE01219D
:100AD000284600F06BFD12B0BDE8F0810024014013
:100AE00000280140002C014008000240B80200200C
:100AF0000D4910B5884202D1012144150AE00B4985
:100B0000884202D10121041504E0094988420AD132
:100B10000121CC03204603F0C5F92046BDE8104072
:100B2000002103F0BFB910BD00240140002801409E
:100B3000003C01400029816802D041F4801101E0AD
:100B400021F48011816070470029816802D041F44E
:100B5000004101E021F4004181607047826822F485
:100B6000E0420A43826070470146002089684907D5
:100B700000D50120704710B50246002054680B0ACA
:100B8000C9B20C401168194202D0002C00D00120DB
:100B900010BD014600208968090700D50120704773
:100BA00038B501211C2003F071F9FF20ADF80000D9
:100BB00000248DF8034003258DF8025069460D4846
:100BC00001F0F0FA0120ADF800008DF803408DF837
:100BD00002506946084801F0E5FA2320ADF800000C
:100BE0008DF803408DF802506946044801F0DAFAA6
:100BF00038BD000000080140000C01400010014019
:100C0000002A4268C9B201D00A4300E08A43426028
:100C10007047000010B542680E4B0C791A400B6803
:100C200042EA04221343436083680B4A1340D1E92C
:100C3000024222434C7943EA44031A438260C26A67
:100C4000097C22F47002491EC9B242EA0151C16214
:100C500010BD0000FFFEF0FFFDF7F1FF70B50724A7
:100C600009290AD9C568A1F10A0606EB4606B4406F
:100C7000A543B3401D43C56007E0056901EB41068C
:100C8000B440A543B3401D430561836BC3F30154D6
:100C9000121B921C02EB82041F22A2409343A1402C
:100CA0000B43836370BD826B491E22F4401242EAFB
:100CB00001518163704770B5072409290AD9C568B5
:100CC000A1F10A0606EB4606B440A543B3401D4316
:100CD000C56007E0056901EB4106B440A543B34098
:100CE0001D4305611F23072A09D2446B521E02EBE4
:100CF000820293409C4391400C43446370BD0D2A93
:100D000009D2046BD21F02EB820293409C439140B4
:100D10000C43046370BDC46A0D3A02EB8202934037
:100D20009C4391400C43C46270BD816841F008014E
:100D3000816070470029816802D041F4A00101E080
:100D400021F4A00181607047816841F00401816055
:100D5000704700210160017141718160C160012112
:100D60000174704770B51E4C214694F83800B1F8F4
:100D7000425006281ED9B4F84A10B4F84C00A1EB32
:100D8000000202F10902122A04D8FFF757FB0022E1
:100D9000144B0AE0884204D2FFF750FB0022124BAA
:100DA00003E0FFF74BFB0022104BFFF730FAFFF791
:100DB0008AFB09E005D12846FFF740FB0C4A0D4BA2
:100DC000F3E70D4951F82000C5EB45116063B0EB26
:100DD000410F03D9C5EB45104000606370BD0000B2
:100DE000540400200000344000003340000035402F
:100DF0006766666666E64B402C90000810B50C4CA2
:100E00002078400713D5FFF7ADFF0A49A08E088070
:100E100008483038018821F010010180001F018846
:100E200041F010010180207820F00400207010BDF6
:100E30005404002040040040F0B4184816494FF410
:100E40009677436C08468A68046815485FEAC25C76
:100E500042F00806007822F008054FEA047415D520
:100E6000002C08DB120714D408B1082811D1BB42AA
:100E70000FDA8E6007E012070BD508B1082808D1F9
:100E8000BB4206DA8D60F0BC05F06EBF002CF2DAD2
:100E9000E8E7F0BC70470000A802002048010020ED
:100EA0001F07002070B506464089204B204C4FF4A8
:100EB0008071002580B362887AB1012A0CD1E18863
:100EC000491C89B2E1803289914205D36580E58071
:100ED000FF2801D0401E708170BD7088228890422A
:100EE00001D9012200E00022184601F0E4F97088DF
:100EF000B18801442088401C80B220808142EBD818
:100F00002580A088401C80B2A080F1888842E3D36D
:100F100001206080A58070BDFFE70022184601F027
:100F2000CAF9A580E58025806580F4E7000C0140C2
:100F3000C4050020FEE70000FCB505464FF6FF762D
:100F400000200C46ADF8006048F205078DF804005B
:100F500020E000BF15F8010B8DF8040001A9084638
:100F600002F0DBF8BDF800009DF8041080EA0120D3
:100F7000ADF800005FF00000BDF800100A0402D5D3
:100F800087EA410101E006EA4101401CADF800108A
:100F90000828F1DB641EDDD26946084602F0A7F896
:100FA000BDF80000FCBD00000246002004E000BFC8
:100FB00012F8013B1844C0B2491EF9D27047000034
:100FC00070B5144A85B01088002413490194009428
:100FD000039420460494138807E00D8B009E35444B
:100FE0000095CD8B019E3544019515889D42F4D026
:100FF000401CC0B28028EED30098411107484180C0
:10100000848001984111064881830183818205B063
:1010100070BD000028070020A8020020DE05002087
:10102000CC04002030B50E4902880A800C4A43885F
:10103000083A13800B1F808818802024151F2C80ED
:101040000020401C80B27328FBD341F211100880AD
:1010500044F64800108047F2480018802C8030BDCC
:10106000202C0140114944F648000880091D46F62D
:1010700048000880091D41F2111008800B48001F2C
:10108000018841F02001018009480021A0F8641086
:10109000A0F86210A0F86010A0F85E10A0F85C1034
:1010A000A0F85A100348418181827047182C0140F2
:1010B000A8020020640000202DE9F04F524B534855
:1010C0000022D97A90F800C080292CF001067DD347
:1010D0001C684F4B01F01F0153F821104D4B0C427F
:1010E000196802D041F0200101E021F02001994669
:1010F0001960484BDFF820B1DFF820A193F8465083
:10110000474B9BF80040B3F90430022C69D1B9F881
:101110000840C4F3C007C4F30024A74261D03D4C8B
:10112000303C94F80380B8F1000F09D0374FB8F184
:10113000010FB7F902700DD0B8F1020F56D120E0BF
:101140000A0553D58A0651D40122E2702CF004021C
:1011500002704BE00E0549D48E0647D55FEA4C7607
:1011600044D4A7BB4380002B09DD4CF0050202707C
:101170000222E2702B4AB2F84420028236E0E2708A
:1011800034E0B0F806C0BCF1000F01D1002B17DC31
:1011900090F80CC0AC4513D107F26667BB420FDC78
:1011A000214FBF895FEA477C0AD45FEA877C07D476
:1011B0005FEA417C04D55FEA816C01D5FF0715D059
:1011C00006704280AAF80020428101E017E00DE09D
:1011D000426182610282E27089F80F208BF8002060
:1011E00004E006704280AAF800204281C3800573A3
:1011F000480960F3CB21C9F80010BDE8F08F0670F4
:1012000042804281F9E70000E40500204C090020FB
:101210008C940008A80200201F0700202401002051
:10122000DE050020480100205C0A00202DE9F0477F
:1012300096B000240C940D940E940F9472B69048BE
:10124000816941F400718161816941F4806181614A
:101250004FF4004002F0ECFD8A4D00212846FFF7D4
:101260002BFB00212846FFF71DFB874E002130464F
:10127000FFF718FB854F0021384600F097F9012051
:101280004FF47041401C8842FCD32846FFF730FCE5
:10129000B1463046FFF72CFC384600F093F94FF486
:1012A0006020CDE912048DF8454001204FF004087C
:1012B0008DF8440010948DF8508010A92846FFF74F
:1012C000A9FC01231A4605212846FFF7F4FC012357
:1012D000022206212846FFF7EEFC01230322072104
:1012E0002846FFF7E8FC012304220F212846FFF7D8
:1012F000E2FC384600F066F9684600F00EFA6148F4
:10130000634E4C300090CDF80C80CDE90164802014
:10131000CDE904404000069080000790202008900E
:101320004FF44050CDE909046946384600F0D8F939
:1013300001212846FFF7C0FA0121384600F036F9AE
:1013400001212846FFF7AEFA47F23051159415985F
:10135000401C15908842FAD301212846FFF7EAFC89
:10136000ADF82C40A04640F2DC5A4FF4007420E067
:101370005046CDF854801599491C15918142FAD3F5
:1013800030880D9908440D9070880E9908440E908D
:10139000B0880F9908440F90F0880C9908440C907D
:1013A00001212846FFF7C6FCBDF82C00401CADF813
:1013B0002C00BDF82C00A042DAD30D98354A40F33A
:1013C000CF1633480A3006830E9941F3CF14448375
:1013D0000F9941F3CF1383830C9941F3CF1CA0F8ED
:1013E00004C0ACF5C05C40F2C371ACF59B7C8C458D
:1013F0000ED2A6F5C856363E8E4209D2A4F5C85480
:10140000363C8C4204D2A3F5C853363B8B4203D3FF
:10141000D18841F48041D180D188490407D41E4944
:10142000028B21F85C2F428B4A80808B88800021C0
:101430002846FFF741FA0021384600F0B7F80021AE
:101440002846FFF72FFA00214C464846FFF72AFAB4
:101450000220C102401C8842FCD32846FFF748FB0B
:101460002046FFF745FB384600F0ACF8FFF72EFAB0
:101470000A493C20087062B616B0BDE8F08700004B
:1014800000100240002401400028014008000240F2
:101490002A0500205C0A0020BC0C00201C0700204C
:1014A000F0B5284B40F22D4643F6FB255C6C264BED
:1014B000B4F5FA5F13DDB4F5FA4F10DC41F6AD1761
:1014C000A4F5FA54674306EBA7364FF4B5777C438F
:1014D00005EBA41475106410C3E9045401E0C3E9DA
:1014E00004651D69D5605C69401A5461106091689B
:1014F000884202DA4942884200DC116010684443A5
:10150000107E0441906A21189162506A814200DD88
:101510009062916A106A814201DB084600E09062A5
:10152000986111684D43117C0D4108412918B2F9A9
:101530001C00884204DBB2F91A00884200DC08B2C1
:10154000F0BD0000480100202801002010B54FF434
:101550000054204600F0ACF8002813D00A4908785F
:1015600040F008000870204600F014F800210748F9
:1015700000F01CF80648C17E012903D10021C17684
:101580000121017710BD00007E06002044000240CA
:10159000600B0020C10002D5024908607047024973
:1015A00048607047040402400000024000290168BE
:1015B00002D041F0010102E04FF6FE7211400160DD
:1015C0007047000001684FF6FE7211400160002173
:1015D000016041608160C1603149314A08399042FF
:1015E00003D1486840F00F0006E02D4A14329042C3
:1015F00004D1486840F0F00048607047284A28321B
:10160000904203D1486840F47060F5E7244A3C32C8
:10161000904203D1486840F47040EDE7204A5032D0
:10162000904203D1486840F47020E5E71C4A6432D8
:10163000904203D1486840F47000DDE7184A7832E0
:10164000904203D1486840F07060D5E7154A111FF9
:10165000904203D1086840F00F0006E0114A1432AE
:10166000904204D1086840F0F000086070470D4ACD
:101670002832904203D1086840F47060F5E7094AC7
:101680003C32904203D1086840F47040EDE7054ACF
:1016900050329042EAD1086840F47020E5E700003B
:1016A0000800024008040240406880B27047000011
:1016B00001460020CA0001D5034A00E0034A12682F
:1016C0000A4200D00120704700040240000002409E
:1016D000002A026801D00A4300E08A430260704792
:1016E00030B5036847F6F07293430C6A8A68224368
:1016F000D1E904452C4322438C692243CC6922431F
:101700004C6A22438C6A22431A430260CA684260D0
:101710000A6882604968C16030BD00210160416093
:101720008160C160016141618161C16101624162A9
:101730008162704710B5114C8CB000212046FFF734
:1017400035FF2046FFF73EFF0D4800900D48002171
:10175000CDE901016420CDE903018020CDE9050137
:101760000791089109910A9169462046FFF7B8FF51
:1017700001212046FFF71AFF0CB010BD58000240AF
:1017800004380140B807002010B501218CB008468C
:1017900002F058FB1E4C00212046FFF707FF2046B1
:1017A000FFF710FF1B4800901B48019000211020FC
:1017B000CDE902018020CDE904100691079108913E
:1017C00009910A9169462046FFF78AFF012202210A
:1017D0002046FFF77DFF01218DF82F1004208DF8A2
:1017E0002D008DF82E100E208DF82C000BA802F085
:1017F00031F80F208DF82C000BA802F02BF80121F6
:101800002046FFF7D3FEFFF795FF0CB010BD000098
:1018100044000240043801405407002030B540F62F
:10182000AA21204AC184838B1488E31A9BB20F2B10
:1018300010D312888283037E002253B11A4BB3F96E
:101840000A30062B05DB194B1B78022B03D0002B2B
:1018500000D1828430BD164B40F68B255B6CA3F221
:101860002D14AC420FD2428B521C92B24283642A96
:10187000F0D364224283B0F924208A4201DA02EBD9
:101880002111818430BD41F29414A342FADBB0F9F6
:101890002430002B02DDA3EB211100E00021818424
:1018A000428330BD28070020640000201F0700206D
:1018B0004801002010B50446B0F9020043F6991122
:1018C00048438113E06840F26662504301EBA03068
:1018D000E060B4F9001043F6991251438A1321696C
:1018E00040F26663594302EBA131216104F0AAFE84
:1018F0006061A18840F6AB2208444010A0F5154174
:101900005539E062914205D9A0F5F851FF39521CD2
:1019100091421DD249F25451884202DDA0F5204087
:1019200002E0A0F5F850FF38206300EB400040F3E0
:101930004F002085B4F924104A42904201DA104643
:1019400002E0884200DD0846E083228461848AE068
:10195000A0F5FE42FF3A41F255518A4214D8A2F650
:10196000AA20206300EB400040F34F002085B4F92B
:1019700024205142E183884201DA084602E0904285
:1019800000DD1046404250E0A0F5D442AA3A8A4217
:1019900015D2A2F6AA20206300EB400040F34F01CD
:1019A0002185B4F924004242E2832084914201DA85
:1019B000104602E0814200DC0846608453E0A0F556
:1019C000AA42543A41F256539A4215D2A2F6AB209B
:1019D000206300EB400040F34F002085B4F9241051
:1019E0004A42904201DA104602E0884200DD084691
:1019F0004042E083218419E0A0F5804241F2545333
:101A00009A4215D2A2F6AA20206300EB400040F3D0
:101A10004F012185B4F92400E0834242914201DA6A
:101A2000104602E0814200DC0846208462841AE00D
:101A3000A0F52852AB3A8A4215D2A2F6AA2020631A
:101A400000EB400040F34F012185B4F92400E0830E
:101A500042422284914201DA104602E0814200DCD7
:101A600008464042A9E7B4F91E00A0EB40208013CD
:101A7000E080B4F92000A0EB402080132081B4F96D
:101A80002200A0EB40208013608110BD012101766F
:101A9000704770471548164A4FF480410078042873
:101AA00021D002F13C03D08A9B88C01A00B22F28B3
:101AB00001DD001108E0002801DD002007E00D4BEA
:101AC000984201DA184602E0402800DD4020938960
:101AD000184400B2884203DC40F26661884200DAB2
:101AE0000846908170479181704700001F070020D1
:101AF000CC040020C0FEFFFF38B54B484B4902889C
:101B00000B889A1A92B20F2A71D30988484C018027
:101B10004FF0FF01E2884FF47A7355044FF496704A
:101B200002D51622009103E0950403D515220091F9
:101B3000014670E0D50402D514220091F8E715059E
:101B400002D513220091F3E7550502D51222009128
:101B5000EEE7950502D511220091E9E7D50502D5FA
:101B600010220091E4E7150602D50F220091DFE76D
:101B7000550602D50E220091DAE7950602D50D2210
:101B80000091D5E7D50602D50C220091D0E71507C4
:101B900002D50B220091CBE7550702D50A2200910E
:101BA000C6E7950702D509220091C1E7D20702D006
:101BB00008220091BCE72289550702D5072200912F
:101BC000B6E7950702D506220091B1E7D20702D009
:101BD00005220091ACE7A27AD20702D0042200913C
:101BE000A6E7A289D40603D503220091A0E719E055
:101BF000140702D5022200919AE7540703D49407F0
:101C000001D4D20702D00122009191E700200346BF
:101C100002460146009002F085FFBDE838400248C8
:101C2000FFF740B938BD0000500A00202807002007
:101C30005C0A0020F0B55948594982880B889A1AE5
:101C400092B29C2A64D30988818056490A88014649
:101C5000002A0B7843F0020156D11646524A1C075F
:101C600015680246127822F0020274D54F4C0746DE
:101C7000E4887F785FEA845C02D547F0010701E0E1
:101C800027F001074770A704477802D547F00207FD
:101C900001E027F002074770670401D4E70703D08B
:101CA000477847F008074770640603D5447844F046
:101CB000040404E01C0603D4447824F004044470B3
:101CC000EC0450D4354C9A07247824F0100423D423
:101CD000324D42782F7A2D78012A45F0100514D024
:101CE000022A16D02D4C042AA47804F1010C0CF021
:101CF000FF0C13D0072A25D0032A23D0052A21D090
:101D0000062A1FD021F0100142E0B90702E0057059
:101D1000F0BD39070029FADB0470F0BDFA0601D4E2
:101D20001A060AD50170022C04D280F802C0BCF158
:101D3000020FF2D341F080012AE021F0100101707E
:101D40008670F0BD877A7F06F7D5032C04D8017022
:101D500080F802C0F0BD0FE05107D8D51906D6D4DF
:101D600043F0800114E002704178CB0701D189076C
:101D7000F0D522F010010BE0E9040BD49907E9D467
:101D8000818AC82902D2491C8182E3E743F00A0113
:101D90000170DFE702708682DCE7000000070020A8
:101DA000280700202A070020A80200205C0A002043
:101DB000094944F648000880091D46F64800088095
:101DC000091D41F6CC4008800348001F018841F0FE
:101DD0002001018070470000182C0140084946F698
:101DE00068000880091D0880091D41F255500880CF
:101DF0000348001F018841F0200101807047000066
:101E0000182C014010B5C28800210AB1032206E057
:101E100002890AB1022202E0428912B10122027053
:101E200000E0017004784FF4804344F6206244B12E
:101E3000012C06D0022C07D0032C01D141808180D7
:101E400010BD4380828010BD41F23331418040F6A5
:101E5000B731F4E730B5B1F86A5000231A240D22E7
:101E6000854202DCB1F9680030BD4D88854202DB55
:101E7000B1F9000030BD01EB82056D88854201DDBE
:101E8000144601E013DA134604EB03024FEA520250
:101E90009A42F0D101EB830231F8231054889288E2
:101EA000521A001B424301EB622000B230BD31F9EF
:101EB000220030BD054920B1086940F0800008616A
:101EC000704703484860034848607047002002405C
:101ED00023016745AB89EFCD06494FF47A70CA6894
:101EE000D20705D0401E0004000CF8D1FF20704737
:101EF00000207047002002400E4A0320A2F150014A
:101F000082F83E00002048810B490886C862C883D9
:101F10000884488490620948816CB1F5206F01DB28
:101F2000A3219162807A002802D0906A4042906298
:101F300070470000640000203405002048010020A4
:101F40000449002048810881C86288620249886289
:101F50007047000064000020C8080020F0B53B492D
:101F600088894A89801A80B20F2866D38889488177
:101F7000CA8937480B3A272A26D28A7822BB826838
:101F8000364B42F480728260324A354C354D1278BD
:101F90005607314A0AD4344E36881680334A12889E
:101FA0001A80334A12882280324A09E0324E36883B
:101FB0001680324A12881A80314A12882280314AA9
:101FC00012882A8001228A702F4B304D19469A7F41
:101FD0000968802A32D302F01F0255F822201142EC
:101FE0002CD0826822F48012184E82601236144679
:101FF0001215B778521C62F38617254AB77093F80A
:1020000016C01778BCF1800F27F0020608D30CF039
:102010001F0C55F82CC011EA0C0F01D147F0020635
:1020200016701A7E802A0DD302F01F0255F8222066
:10203000114207D144F400218160F0BD826842F46E
:102040008012D1E724F40021F6E700001C070020ED
:10205000A802002048010020C4040020C60400207B
:10206000C8040020CA040020B4040020B6040020E4
:10207000B8040020BA040020BC040020BE040020E4
:10208000C0040020C2040020E40500208C94000855
:10209000CC04002070B5204881890289891A89B250
:1020A0000F292FD3818901811C4B1D4819465D7A68
:1020B00006681C4C096846F00402802D07D305F021
:1020C0001F0554F82550294201D126F00402026070
:1020D0009A7B802A17D302F01F0254F82220114263
:1020E00011D1026822F002020260DA7A802A0ED34D
:1020F00002F01F0254F82220114208D1016821F099
:102100000801016070BD026842F00202ECE701685C
:1021100041F00801F5E700001C070020E40500205D
:10212000A80200208C940008F0B51D4C1B4A4FF00B
:10213000010C94F83B5094F80AE0144692F83C30B5
:1021400094F838402B43651CEEB2154D95F83D7060
:102150000025BEF1FF0F0AD0BEF1000F06D18B4261
:1021600013D155700C2C01D282F83860F0BD834237
:1021700002D182F801C0F5E78B42F7D15570B8075C
:1021800009E000BF82F83850F0BD8342FCD1F8432B
:1021900082F801C080070028F4D0F0BD540400206C
:1021A00048010020F0B5CA78002502F00F03D206DE
:1021B00001D58A7813430A784FF00F0E12F0FF0F03
:1021C0004FF001021CD004680F8802FA05F6374070
:1021D000B74211D14FEA850C0EFA0CF724EA070733
:1021E00003FA0CF43C43CF78282F02D0482F02D0BA
:1021F00002E0466100E006616D1C082DE4D3046036
:102200000C88FF2C1ED944685FF0000606F1080711
:1022100002FA07F50F882F40AF420FD14FEA860C24
:102220000EFA0CF7BC4303FA0CF73C43CF78282F87
:1022300000D14561CF78482F00D10561761C082E6A
:10224000E4D34460F0BD0000F0B5144C002801DA7E
:10225000E36900E06368420D120185B2C0F30157E3
:102260009540C0F30346032F05D0C2020AD50322CE
:10227000B240934307E023F07062636823F0706319
:10228000636002E0AB4343F0706201B12A4300286F
:1022900001DAE261F0BD6260F0BD000000000140C3
:1022A0000246002092680A4200D001207047416136
:1022B0007047016170470AB1016170474161704721
:1022C0000F4A104B92F838105B5C834201D1012019
:1022D00004E00D4B5B5C834203D1002082F83A009E
:1022E00070470A4B5B5C834201D18120F6E7084BC3
:1022F000595C814201D18020F0E70320EEE7000025
:102300004801002044990008569900084A9900089D
:102310005C9900080A4810B501784FF000024C079C
:1023200008494FF0FF0389684FEA017105D500297C
:1023300001DA827210BD837210BD0029FBDBF8E761
:1023400048010020A8020020F0B5194E194C0022C7
:10235000E31CA6F1060CB75CA518ED78FF5C0D43F5
:102360000F43BD421FD01CF80270FF5C0F43BD42FB
:1023700019D015460023A618F6780E43C6545B1CE8
:102380001CF80220DBB2062BF5D3C17881700179ED
:10239000C17000214218491C15711CF80550C9B2C2
:1023A0000629F7D3F0BD521CD2B2032AD3D3F0BD15
:1023B0001E9000085404002010B502460021064B70
:1023C00006205C186478944200D10846491CC9B2C2
:1023D0000629F6D310BD000048010020214810B5A1
:1023E00090F8671000222048012936D11F498988BA
:1023F00099BB1F491E4B4C6C40F6B831B3F86E3098
:102400008C4227DD1B49097821BB90F82711491C14
:10241000C9B280F82711C8291CD380F827210146AA
:10242000D0F82C4191F82811A34203DD052908D2E8
:10243000491C01E041B1491E80F82811C9B20529A3
:1024400002D3012180F82611191B074C303CA162F0
:10245000C0F82C31B3F5FA6F03D280F8262180F84A
:10246000282110BDBC0C0020A8020020DE050020A1
:10247000480100201F0700204FF4C042C260002125
:1024800081620E22028241F26202426108220283CC
:102490004FF46042428381834FF07842C0E90821C3
:1024A00040F6C41101807047B0F90010B0F9022065
:1024B000891A41604269037E4A431A41836A134480
:1024C0008362426A934200DD8262836A026A9342B7
:1024D00000DA8262C268836A4A43017C0A410B4186
:1024E000D118B0F91C208A4201DA10467047B0F9C1
:1024F0001A008842FADC08B27047000010B5144890
:102500001449B0F88C200B889A1A92B2B2F5437F26
:102510001DD90988A0F88C10B0F88A1020F8581F2F
:10252000002242860C480D4CC2888280C180C3893B
:1025300083812489891AA4B2C4818160E11A01616E
:10254000074A818AC182928A8282511A816110BDB2
:102550004801002028070020840C002034050020BA
:102560006400002009480A49B0F8AA200B889A1A8A
:1025700092B241F684639A4206D3098820F8AA1FD2
:10258000418881800021418070470000480100207F
:10259000280700200D480178C90702D00C49098896
:1025A00001E04FF6FA71C165094901201039088030
:1025B00007482438018841F0010101800448183897
:1025C000018821F0180101807047000048010020B7
:1025D000240400400A49D1F8902012B1521EC1F8DB
:1025E000902031F88A2F521C21F81A294A6A521C6D
:1025F0004A628A8F521C8A8701F8380C70470000A3
:10260000480100201CB52D4890F83B3090F83C2044
:10261000934252D000248DF8044053408DF800308E
:102620009DF800300122012B08D09DF80030022BCC
:1026300009D09DF80030042B0AD00DE01F498DF819
:102640000420443108E01D498DF80420463103E0A0
:102650001A498DF8042048319DF80420012A2CD114
:1026600090F83D309DF80040154AA34217D090F8ED
:102670003E309DF80040234208D0B0F84C30A0F81E
:102680004A300B881488E31AA0F84C3090F83830A0
:102690002BB1B0F840301488E31AA0F84230128809
:1026A0000A80A0F8402010F83E1F9DF8002011433A
:1026B00000F801199DF8001001701CBD54040020A1
:1026C0002807002070B5344D40212846FFF7E8FD6B
:1026D000840080212846FFF7E3FD44EA4004A91561
:1026E0002846FFF7DDFD0443E1B22C4C94F870500E
:1026F0008D4250D04D4084F87010012D03D0022D32
:1027000001D0042D47D194F87400A84384F87400D4
:1027100094F87320AA420FD084F8735094F8722072
:1027200001238B401A4207D11A4384F8722094F88F
:102730007110491C84F8711094F87110042928D381
:1027400030B1012811D002280FD004280DD012E09A
:102750001348C18821F04001C1802078002184F80D
:102760003B1020F06000207005E0217841F020014E
:10277000217084F83B000B4994F83B0091F8272026
:10278000904204D081F8270007492020087000F00B
:102790000DF884F84C5070BD001001404801002035
:1027A0005C0A0020BC0C00201C07002070B50D4DF9
:1027B00040212846FFF774FD840080212846FFF75A
:1027C0006FFD44EA4004A9152846FFF769FD04435C
:1027D0000548072100F8704F017100214170817098
:1027E000C17070BD001001404801002070B5344830
:1027F00090F83A10CA43920761D001F0030280F8C2
:10280000392090F83D305B061B0E80F83D30012AE0
:1028100001D0812A02D15B1C80F83D300278D207BA
:102820004DD0DBB203F00102C3F34004A24246D113
:10283000B0F84E400025641CA0F84E40204CA0F893
:10284000505090F83E60A47AB24202D080F83E2008
:102850000DE0A607B6EB837F02D080F83F5006E07C
:1028600090F83F30642B02D25B1C80F83F3090F828
:102870004030642B0CD25B1CDBB280F84030022B62
:1028800006D204F00103934202D1022280F84020D4
:10289000012901D0002912D190F83820C16D00EB38
:1028A000820291610163D0E906121144D0E9082344
:1028B0001A441144826A1144C26A1144416370BDD2
:1028C00048010020FEE700002DE9F04F00BF002086
:1028D0009E4E9F4AA6F51271A6F5BE79A6F1440B4D
:1028E00006F1440E804601F5E074A1F1780301F58C
:1028F000457A1D5C15F0C00706D0402F51D0C02F7F
:1029000077D0802F76D004E115F01F0504D0154450
:1029100040F080072F7201E082F80880012826D05D
:10292000022824D0032822D0042820D008281ED032
:1029300010281CD0874D55F820C0DCF8005054F802
:1029400020703D40CCF80050824D55F820C0DCF896
:10295000005056F820703D43CCF800501D5CAD0689
:1029600059F820502F6813D53AF810C03EE051F8BE
:1029700020502F6854F820C007EA0C072F6051F848
:1029800020502F6856F820C047EA0C072F60E5E773
:10299000DFF8B8C10CF1F00C5CF820C007EA0C07B6
:1029A0007EE015F01F0504D0154440F080072F721B
:1029B00001E082F8088001281DD002281BD00328DE
:1029C00019D0042817D0082815D0102813D0614D2D
:1029D00055F820502F6854F820C007EA0C072F60E4
:1029E0005C4D55F820502F685BF820C047EA0C0773
:1029F00056E00BE056E051F820502F6854F820C004
:102A000007EA0C072F6051F82050ECE715F01F057E
:102A100005D0154440F0800785F8217001E082F868
:102A20002180012825D0022823D0032821D0042882
:102A30001FD008281DD010281BD0464D55F820C0A7
:102A4000DCF8005054F820703D40CCF80050414D67
:102A500055F820C0DCF800505EF820703D43CCF8FB
:102A600000501D5CAD0615D53A4D3AF81070CC35C6
:102A700014E051F820502F6854F820C007EA0C07E2
:102A80002F6051F820502F685EF820C047EA0C07ED
:102A90002F60E6E72D4D3AF81070E03D55F82050D4
:102AA0002F6036E015F01F0505D0154440F0800773
:102AB00085F8217001E082F82180012830D00228B9
:102AC0002ED003282CD004282AD0082828D010285B
:102AD00026D0204D55F820C0DCF8005054F8207066
:102AE0003D40CCF800501B4D55F820C0DCF800509C
:102AF000164F883757F820703D43CCF800501D5CC6
:102B0000AD06B1D4114F3AF81050E03F57F820709D
:102B10003D60401CC0B21128FFF4EBAEBDE8F08F61
:102B200051F820502F6854F820C007EA0C072F6096
:102B300051F820502F68DFF814C00CF1880C5CF8B5
:102B400020C047EA0C072F60D9E70000189700085B
:102B5000E4050020149500084FF40771C1824FF47A
:102B60005861018340F6145181837047F0B5C48ADF
:102B7000B0F900608681B0F90250C581B0F9043027
:102B80000227002101220382AB4204DBB54202DDB1
:102B9000C78042810CE0B34204DBAE4202DDC78055
:102BA00041811CE09D4205DBB34203DDC2804781C9
:102BB000018115E0B54204DB9E4202DDC280418105
:102BC00005E0AE4205DB9D4203DDC1804281078105
:102BD00006E09E4204DBAB4202DDC18047810281F8
:102BE000C388458900EB430700EB4505BB89AE89E7
:102BF0009B1B0FFA83FEA0F812E00689AB8900EB5D
:102C0000460CBCF80CC0A3EB0C038382B0F918305F
:102C1000B7F90CC0A3EB0C0CB4EB4C0F04DA80F842
:102C20002010A3F1A10113E0A64503DD80F82010D8
:102C3000B9890BE026B1012E04D0022E10D004E099
:102C4000062100E0052180F82010A989091B6D31BB
:102C5000418309B2B1F5586F04DB5B1E438304E086
:102C60000421F0E7002900DC4283418B8183F0BD21
:102C70000B49002288760A62CA614A62094A32F91F
:102C8000103002EB40028B62B2F90220CA62064A9F
:102C900032F810000882A1F86000A1F862007047C5
:102CA000F80100206E990008629900082DE9F05F94
:102CB000FD48FE4982880B889A1A92B20F2A44D3A3
:102CC0000988FB4A8180814611880124F948FA4E1F
:102CD000002579B3491E1180C573F84A85620168E1
:102CE000B2F902204F0742F6AA2318D4F78847F416
:102CF0000057F780F14E3678B60709D5866826F07A
:102D000080068660A0F87C5080F87E5080F87F5066
:102D1000CE0404D480F8F040C0F8EC5003E080F812
:102D2000F0504E0707D49A4205DB80F8F440A0F833
:102D3000F25004E010E080F8F4504E0703D49A42B9
:102D400001DBC90703D080F81151BDE8F09F80F87E
:102D50001141A0F81251F8E78046B0F8181143F677
:102D60009820814202D2491CA8F8181101F0F0FE07
:102D7000D34FDFF834B397F85000ABF11C0B10B110
:102D8000FEF79AF905E09BF8001021F001018BF89D
:102D90000010FFF723FB00F0D7F9CA4841F26802A0
:102DA0004FF40061406C904201DBC74A04E0B0F58B
:102DB0007A6F02DAC44A121D116097F85110DFF8D9
:102DC000F4A2C24BC24FC907AAF1300A3AD0997B8C
:102DD000802933D398F8002092072FD498F80F2039
:102DE0008AF80720B54A514692F800C02CF0020C30
:102DF00082F800C0ABF80250CBF814509BF800C02A
:102E00002CF0010C8BF800C0B279520611D48A89DB
:102E1000B2F5FA7F03D2521CAAF80C2012E040F659
:102E20003C72904201DD002013E108208AF8044042
:102E30000FE10D710020AAF80C500AE18AF8045045
:102E4000AAF80C50D8F80800010501D5082000E1C7
:102E50009B4991F83FE05FEACE7149D09B4B98F8CF
:102E60000F208AF807205B7A4146802B4CD30B78E1
:102E70005B0735D4F3889B0405D500BF20F0200004
:102E8000C8F8080034E0ABF80250CBF814509BF8B7
:102E900000C08E4B2CF0010C8BF800C040F02000DD
:102EA0008860D87D80280AD300F07F0C1B684FF023
:102EB000004020FA0CF0034201D10C7100E00D71CA
:102EC0000879C00702D15FEA8E7005D50320032A76
:102ED00001D08AF80A40BCE00020C8F82850B8E0C9
:102EE00020F02000C8F80800F08820F40050F0809E
:102EF00098F82601444601280BD0714890F86300E9
:102F000048B1FDF799FF0FE00A6842F004020A6039
:102F1000B4E709209DE0A068C10502D520F00800B3
:102F200001E040F00800A06094F846304FF4804182
:102F3000E3B143F69912012B1FD0881E022B2FD02C
:102F40003B78C3F38103012B2FD0022B2DD0A4F8A3
:102F50001411604890F85E0004281ED0A4F84410B4
:102F6000574890F87000012822D031E043F21E50FB
:102F7000A4F8140143F2333014E0387842F6CC431D
:102F8000C0F38100012806D0022804D043F2EB10E0
:102F9000A4F8140101E0A4F81431A4F84420DFE7F8
:102FA000A4F81401A4F84400DAE7A4F81401D0E767
:102FB0003878C0F3810242F26660012A0FD0022AFB
:102FC00010D041F6E12200BFA4F81421A4F8440077
:102FD0009BF80020D20708D0BBF8022007E0A4F835
:102FE0001401F3E74FF40052EEE734488288A9F861
:102FF000122010B2B4F944205043C0F38F3250462F
:10300000AAF814208A4200D9818233490978C90676
:1030100005D5828A41F233318A4200D281822189E8
:10302000C1F3C002C1F300218A4205D1828A40F671
:10303000CC418A4200D98182B17AC90700D0858209
:10304000BAF81400A06200287FF7EDAE234805709F
:10305000022099F81A1099B9022841D080B1194973
:103060000B789C0608D5B479640605D51A4C2478EB
:10307000E40964F386130B70F18821F40A61F1808E
:103080001049496C4E290ADBF1880B0607D521F05F
:103090008001F18009490B7823F002030B7089F855
:1030A0001A0088F80F0050E6680900202807002061
:1030B0002A070020A80200205C0A0020DE0500206C
:1030C000BC0C002048010020100C0140E405002049
:1030D000CC04002064000020000700203C070020F2
:1030E000398F0029BBD143F698213987B7E770B5EE
:1030F00000230C8863F30F02012505FA03F634421E
:1031000006D0C3F10F0605FA06F1114361F30F0271
:103110005B1C102BF1DB028070BD70B500230C78B6
:1031200063F30702012505FA03F6344206D0C3F122
:10313000070605FA06F1114361F307025B1C082B31
:10314000F1DB027070BD0000F0B51F4890F86630EA
:103150001E48012B816821F4006232D11C4BDE88AD
:1031600074062ED41B4D0F054FF00004B5F9025024
:103170001ED4194A526C642A11DC40F6386295421A
:103180000DDAB2040BD4027852070ED4B0F8D42072
:1031900040F6B835AA4203D2521CA0F8D420F0BDA4
:1031A00041F4006181605C81F0BDA0F8D440F0BDC5
:1031B00041F2CD018D42FADD997AC907F7D18260DB
:1031C000F3E78260F0BD0000BC0C0020A8020020E4
:1031D0005C0A0020DE05002048010020F0B5364DD5
:1031E000364F044695F83B0097F83B102378084388
:1031F000EE1C6278834205D1E0781146FEF794FF19
:10320000207908E094F802C084450CD1E17810469A
:10321000FEF78AFFE07905F82F0F2878805D687047
:10322000287BE877F0BD82421DD161461846FEF743
:103230007BFF95F84E1095F83B00814207D1B97A93
:1032400009B1A17900E0617985F82F101EE0697855
:10325000012901D0A17922E0617927E0297841F0A4
:103260000401297012E0E1788142DBD11946604601
:10327000FEF75AFF95F84E1095F83B0081420AD1AF
:10328000B97A09B1617ADFE7217ADDE715F82F1FF6
:10329000895D6970C5E76978012906D0617A85F88A
:1032A0002F10B97A0029F1D1D8E7217A85F82F10AB
:1032B000B97A0029EAD0D1E754040020480100205F
:1032C0000B48017821F0020100F8381B002100F8BA
:1032D00018194177817733218185418508214184FF
:1032E000012100F81F1C034880F8391070470000C6
:1032F00054040020480100200D4900B50B4851F846
:10330000012F40F8032F8988818008480121093066
:10331000FFF71AF8054802211330FFF715F80348A4
:1033200004211D305DF804EBFFF70EB854040020B3
:1033300048010020094944F648000880091D46F666
:1033400048000880091D41F2111008800348001F41
:10335000018841F02001018070470000182C0140D5
:103360002DE9F047664C674B0025A0780126654A99
:10337000103305287ED2DFE800F00313113E110060
:10338000108820F0010010801D805F480580001F1C
:103390000580001F0580FFF7CDFFA670BDE8F08710
:1033A000594941F244401C390880574945F65800B4
:1033B00024390880091D47F258000880524920200E
:1033C000283908800020401CC0B27328FBD3FFF7C7
:1033D000B1FF4C4984F85C502C3147F6906008806E
:1033E0004848143006801D80108840F0010010808D
:1033F0000220A070D2E700215FF0010004EB41023F
:1034000004EB4003B2F85020B3F850309A4200D297
:103410000146401CC0B20628F0D33C48405C84F80A
:103420003900FFF74DFF1D2000F0F3F900F076F8AA
:10343000374E38484FF4807996F83B10012904D074
:1034400002291BD0042930D047E040218046FEF7F6
:1034500027FF870080214046FEF722FF47EA40070A
:1034600049464046FEF71CFF074347F0010084F839
:103470003B0000E03DE0224809302CE0402180463E
:10348000FEF70EFF870080214046FEF709FF47EA5E
:10349000400749464046FEF703FF074347F0020056
:1034A00084F83B001648133015E040218046FEF7B3
:1034B000F7FE870080214046FEF7F2FE47EA40070C
:1034C00049464046FEF7ECFE074347F0040084F807
:1034D0003B000B481D3002F09FFF94F82F0086F848
:1034E00038001D2000F0ABF90420A0700A480570D8
:1034F00054E7108820F0010010801D80A5704DE772
:1035000054040020000800403C2C01402490000896
:1035100048010020001001401F0700202DE9F04164
:10352000344C14F82F0F344DE07240212846FEF73A
:10353000B7FE860080212846FEF7B2FE46EA400626
:10354000AF1539462846FEF7ABFE0643207BF1B2A5
:103550002F3C814215D084F83C0040212846FEF7DC
:103560009FFE860080212846FEF79AFE46EA400626
:1035700039462846FEF794FE064384F83B60FFF781
:1035800041F81E4D95F83B00012827D0022828D08D
:10359000042829D0174894F83B102730085C04F819
:1035A000300F14F80109FEF707FF04F82F09A87A75
:1035B00000B10120607001F063FB94F84E0094F8B4
:1035C0003B10884206D094F83800062802D2401CEE
:1035D00084F8380084F84E10BDE8F08105480930C1
:1035E00004E00448133001E002481D30BDE8F0411A
:1035F000FFF7F4BD540400200010014048010020F2
:103600002DE9F041524991F87200AA287ED191F833
:10361000730055287AD14F4C00200A5C2254401C7C
:10362000C0B27428F9D34C4E2069C6F80100A08AB4
:10363000A6F80500D4F81600F060D4F81A0030613E
:10364000D4F81E001234706102F08CFE4349608A87
:10365000888102F0A1FE207D123CC007307802D0A4
:1036600040F0040001E020F004003D4930704FF4C8
:1036700080403C4D886114F8280F85F82000608B4D
:103680006880A08BA880E08BE880208C2881608CEB
:10369000354F688194F8240087F8D20014F8011C93
:1036A000304686F83B100026C0F89460FFF724FEF1
:1036B0002E48A18E0183E18E4183218F818394F86E
:1036C0004210283C012908D0022901D0032909D041
:1036D000297821F00C01083107E0297821F00C014C
:1036E000091D02E0297841F00C01297094F86E2040
:1036F000012162B1012A01D0022A0BD087F84610BD
:1037000094F864301A4A4BB1518108E014E087F80C
:103710004660F5E7022287F84620F1E7568194F8E3
:10372000701001290AD094F86D1051B101290BD005
:103730004FF48051A0F87610BDE8F08144F21C717E
:10374000F8E74FF40051F5E741F25551F2E7000078
:1037500000FC0008BC0C0020480100206400002090
:10376000540C0020CC040020A802002034050020C6
:103770005C0A00207CB50121082000F087FB4FF493
:103780008070ADF8040010248DF8074001208DF8FA
:10379000060001A91548FEF705FD0121092000F0EA
:1037A00075FB01211248FEF74FFD0820ADF800001F
:1037B00004208DF803000F4E03258DF80250694652
:1037C0003046FEF7EFFC08213046FEF770FDADF8FD
:1037D00000408DF803408DF8025069463046FEF7F0
:1037E000E1FC10213046FEF762FD7CBD0014014073
:1037F00000023000000C0140FEE7704700F01F029D
:10380000012191404009800000F1E020C0F88011C2
:10381000704700F01F02012191404009800000F133
:10382000E020C0F88011704700F01F020121914094
:103830004009800000F1E020C0F80011704700F05E
:103840001F02012191404009800000F1E020C0F8F2
:103850000011704770B50F23C47801780122F4B1CC
:10386000144C2468457804F4E064C4F5E064240A48
:10387000C4F10406E3408478B5401C402C4301F1B8
:10388000E021230181F80034007800F01F018A4014
:103890004009800000F1E020C0F8002170BD01F077
:1038A0001F0082404809800000F1E020C0F880211C
:1038B00070BD00000CED00E00249084302490860B9
:1038C000704700000000FA050CED00E02DE9F05F04
:1038D00000261D20FFF792FF6C4CDFF8B4B1A4F175
:1038E000B000A77E90F83810DFF8A8E1DFF8A8A1B3
:1038F00000258F427ED0E776A176626A036B5A4339
:103900004FEA12499BF80820120702D51EF8012041
:1039100000E00A4694F812C0BCF1010F09D004EB94
:103920004206B6F902C0C4F828C0B6F90460E662DF
:103930000CE043F6FF7CC4E90A5C90F83DC05FEA06
:10394000CC7C01D012B102E0052A00D1012600EBA7
:1039500047074FF0804CBF893F04B7FBF3F3E361A7
:10396000476BBCFBF7F7276294F813C0BCF1000F5C
:1039700006D0BCF1010F05D03B4403EBD3735B10C1
:10398000636201E03B466762DFF810C14FF6FF77E4
:1039900007EA8307ACF808709AF8007090F80A807C
:1039A00090F83DC0082F08F003070CF0030C05D079
:1039B00067450BD1B8F1000F05D008E0674505D089
:1039C000B8F1000F03D05B42636200E06562C6B1EC
:1039D000636A002B03D006DD228D05E00AE0304B40
:1039E00033F8122000E0A28DA4F86020227822F0A3
:1039F000200222709AF80020042A07D0082A05D055
:103A000012E0B4F8603003EB0902EDE780F84050B3
:103A100065629BF80800000701D51EF801102048D8
:103A200030F81100A4F860001E49606A09883E3130
:103A30004843B4F8601001EB204006B21D20FFF7A8
:103A4000F3FE606A002807D021784FEA81600ADD22
:103A5000002804DAA08D09E0B4F8600006E0E06A0E
:103A6000B04208DB0CE0002802DA208D208208E05A
:103A7000A06AB04204DD208241F02000207000E006
:103A80002682257565752586BDE8F09FF801002022
:103A9000A8020020509900081F070020340A0020C7
:103AA000629900082404004043184FF48042934276
:103AB00010DD904202DD104600210BE0914202DD54
:103AC0000020114606E08003B0FBF3F000B2C0F521
:103AD000804109B241EA00407047F0B54FF46A7383
:103AE0000022C3600E24826204824FF483450826BC
:103AF0004561068343F6FF774283878340F2492E70
:103B00004FEA873CC0F808E0C0E9082CCB608A6225
:103B10000C824D610E834A838F83B4208860C1E993
:103B2000082CF0BD002181620949C1600E2101828B
:103B30004FF6BF514161082101834FF44041418359
:103B400043F6FF71818309070162024941627047B0
:103B5000638A010000C0FF0F064941F6A260088099
:103B600005480168054A01F4E06111430160BFF3B3
:103B70004F8FFEE7442C01400CED00E00400FA05F5
:103B800038B501210D2000F081F94FF4E060ADF867
:103B9000000018248DF8034003258DF80250694673
:103BA0000D48FEF7FFFA4FF46040ADF800008DF8C5
:103BB00003400A4C8DF8025069462046FEF7F2FA9F
:103BC000A014ADF8000048208DF803006946204697
:103BD000FEF7E8FA38BD000000080140000C014083
:103BE0002DE9F0410121CE028CB0304600F04EF9B3
:103BF000DFF86C81404601F0BBFC08A801F0E4FE50
:103C00004FF45860ADF824000024ADF82040202087
:103C1000ADF822000125ADF826408DF8285008A9FE
:103C2000404601F083FE0021404601F0D6FE4FF6EB
:103C3000FF71404601F0DBFE01220021404601F009
:103C400067FE0121404601F04FFC04A801F067FC2B
:103C5000ADF81060A802ADF81200ADF81440A22033
:103C6000ADF816002803ADF81800ADF81A40ADF80D
:103C70001C4004A9404601F041FC6027ADF80070EB
:103C8000ADF80440ADF80840ADF80C40ADF8024086
:103C9000ADF80640ADF80A40ADF80E406946404622
:103CA00001F026FD6946404601F068FD6946404640
:103CB00001F0AEFDADF8045040F61450ADF80070C0
:103CC000ADF80600ADF80840ADF80C40ADF8025074
:103CD000ADF80A40ADF80E406946404601F0DCFD03
:103CE0000121404601F024FC0821404601F040FD3E
:103CF0003146404601F082FD0821404601F0C6FDF4
:103D00003146404601F0FAFD7021404601F003FEC5
:103D100018208DF82C008DF82D408DF82E408DF850
:103D20002F500BA8FFF796FD0D480C30018841F08D
:103D3000800101800A481430018841F001010180AE
:103D4000001F04800121404601F0FCFB8DF8285043
:103D50000121404601F000FC0CB0BDE8F0810000FC
:103D6000002C0140704740F21341416008218160FE
:103D70008621C1604FF480410161494241610021C7
:103D80000162C162704701627047000010B501888E
:103D90004288891A09B20183B1F5005F02DBA1F5FF
:103DA000804104E011F5005F02DC01F580410183F0
:103DB000B0F9182041685143C1618368846A534354
:103DC000C2681B12624303EB2222036A1A441144A5
:103DD00002628A13426241698A4203DB01698A42B4
:103DE00000DC11468A1AC0E90A21028E4FF40373DF
:103DF000594302EBA13202860B4A1278082A04D1F9
:103E00000A4A936F03EBA1319167B0F93010B1F515
:103E1000804F02DDA1F5804103E0002902DA01F5BF
:103E20008041018610BD00001F070020700A00209D
:103E3000034A516821F4404101435160704700003A
:103E400000100240044A0029516901D0014300E0FA
:103E5000814351617047000000100240044A00296C
:103E6000D16901D0014300E08143D1617047000076
:103E700000100240044A0029116901D0014300E00A
:103E8000814311617047000000100240044A00297C
:103E9000916901D0014300E08143916170470000C6
:103EA00000100240044A0029D16801D0014300E01B
:103EB0008143D160704700000010024030B52449B2
:103EC0004A6812F00C03234A03D0042B01D0082BBC
:103ED00026D002604A680F231F4C03EA1212A35C2B
:103EE0000268DA4042604B68072505EA1323E35C69
:103EF00022FA03F383604B6805EAD323E35CDA40DC
:103F0000C2604B68032403F4404104EA933303EB9B
:103F10009161114B1B1F595CB2FBF1F1016130BD86
:103F20004A680E4B1A404B68140103F4803303D5E2
:103F3000C2F38342113202E0022404EB924213B135
:103F40004B689B0301D5064B00E0024B5A43C0E788
:103F50000010024000127A000400002000003C081B
:103F600000093D002DE9F041274CA61540212046CF
:103F7000FEF796F9850080212046FEF791F945EA83
:103F8000400531462046FEF78BF90543EDB240214E
:103F90002046FEF785F9870080212046FEF780F94C
:103FA00047EA400731462046FEF77AF90743F8B260
:103FB000A842DBD140212046FEF772F9870080211C
:103FC0002046FEF76DF947EA400731462046FEF7E6
:103FD00067F90743F8B2A842C8D140212046FEF74E
:103FE0005FF9870080212046FEF75AF947EA40072B
:103FF00031462046FEF754F90743F8B2A842B5D13E
:104000002846BDE8F08100000010014010B50268AC
:10401000416802FB02F301FB01330D4CA34211D9AD
:104020001B0E0E3B0B4C9BB212B234F8133009B28C
:104030005A43594342F38F3241F38F31C0E9022191
:10404000012102E0C0E902210021017410BD00003D
:10405000E10BBF0EC48C00082DE9F05FFA48FB4964
:1040600002880B889A1A92B20F2A7DD30988F84DDC
:1040700001802946A889C988420703D4820701D450
:10408000C20702D041F4007101E021F40071E9801F
:10409000010701D4C00603D5E88840F0010002E022
:1040A000E88820F00100E880E948FDF7ABFEDFF882
:1040B000A4B3BBF93A00B0F5804F01DA401C01E02F
:1040C0004FF48040DFF89093ABF83A0041F6CC41D2
:1040D000D9F84830DFF884838B4205DDD8F8080032
:1040E00020F01000C8F80800DD49DE4E00240888E2
:1040F00028B1401E088088F80F40347026E0E88818
:1041000041041AD4A989CA0617D4090715D401068F
:1041100013D4810611D401050FD4410603D5D24929
:104120000978090609D5410707D4C10505D4010757
:1041300003D4810401D4C00608D5CC4888F80F40C8
:10414000CB493470C4830C8080F82A40B8F83E0014
:10415000C849DFF824E358B1401EA8F83E000878AB
:1041600020F00200087000E0E7E088F80F400AE065
:10417000087840F0020008703078012804D19EF8D9
:104180000000062800D134703078DFF8F0A2012753
:104190000A2871D2DFE800F0F1D105D1F0EFD1703B
:1041A000EEEDAE4D40F62823303D40F6CC4E288B48
:1041B000401C82B2A8482A83406C984201DA2C83C2
:1041C00012E0DBF80CC0F4450EDBB1F9041043F645
:1041D0009913994208DBB2F5FA7F05D39AF80020CB
:1041E00012B92C838AF80070A54B198851B16979EE
:1041F000491CC9B26971022904D3A2496C710A88A9
:10420000521C0A8098F80F10092919D0DFF878920B
:1042100002297DD0A8F830414FF44052CAF87C20E2
:10422000CAF87820B8F84010B9B141F28832214676
:104230002C83904226DA9AF80020012A1DD021E032
:1042400081484430FEF718F9FDF756FE8248406C6D
:10425000E86241F27C50E861EBE2BAF81410A8F889
:104260003010DAF82C10CAF83410DAF82810CAF82E
:104270003010A8F8407035E027E282488AF8001034
:104280000180198099F8682040F63A20012A0CD064
:10429000C8F8D81088F8EA106962B8F9301001F24D
:1042A0001D52824217D8102316E098F8282102B92F
:1042B0007649C8F8D81088F8EA70B8F9301001F2D9
:1042C0001D528242B8F8D80000B201D8102300E095
:1042D0002023102202E020231022002000F02EFCD8
:1042E000A8F8300099F86800694901285A484FF445
:1042F000927315D0406C40F2DC52904203DABAF966
:104300000A209A4215DBB8F84020521C92B200E015
:104310001EE040F6C413A8F840209A4209D20EE0ED
:10432000426C40F2DC50824207DABAF90A00984245
:1043300003DA347088F8EA404C83BDE8F09FDBF87C
:104340000C20002AF9DC42F6E0629042F1DAF4E750
:10435000414AB2F8AE10A1F16403B3F5967F01D8DB
:10436000AB785BB1B1F5C87F14D9A97801290BD01E
:1043700010E035E111E15BE156E15EE14549AF70E6
:104380000B8823F4805304E04249AC700B8843F45B
:1043900080530B80B8F8301140F6B83399420BD2F5
:1043A000DFF8A4C0ACF11C0C9CF800C05FEACC7C28
:1043B00002D1491CA8F830111FFA81FC40F2DC51EF
:1043C0008C4502D842F6CC4303E0A8F8303143F2E2
:1043D0006663CAF87C30E8626F722F49A8F84040E3
:1043E00088F8EA404A7FDAB1C87F0F4650B3B8F880
:1043F0002800B8F9301000B20A23052200F09EFB15
:10440000A8F83000FC777C77B8F91601B8F91411D8
:1044100088427BDA99F84D10A9B100F102008DE0D5
:1044200099F86810012908D1DBF80C1040F23332FA
:10443000D14202DC98F8261181B398F8461002297F
:1044400033D036E067E06EE06809002028070020DE
:104450005C0A00203405002048010020A80200204A
:104460002C0700201F07002000070020F80800206C
:104470001E000020DE050020200700206400002030
:104480002000002022000020BC0C002034F3FFFF9D
:10449000DC090020442C0140840C0020FFE7A3230A
:1044A000B8F930101A4670462BE099F86D100229C1
:1044B00015D0FF4900B200BF01F01AFDA8F8E400D2
:1044C000D8F8281000B2814200DA084600B2E8822B
:1044D00099F84D203AB1B8F93010362310E0F4497C
:1044E00000B2B031E8E7F34A44F2506640F24713B5
:1044F000526CB2420BDD99F8681041B1B8F9301036
:10450000052200F01BFBA8F830007DE70DE0B8F9AC
:1045100030103622F5E740F26660A8F8300088F8DF
:104520000F40347070E7083008E00ADDA979491CB3
:10453000C9B2A971022906D3AC71401EA8F81601B0
:1045400001E0A8F81611DAE91E12914208DA99F88A
:104550004D2012B101F102010CE001F1080109E066
:104560000BDDAA7902F10102D2B2AA71022A06D3A6
:10457000AC71491ECAF8781001E0CAF87820B8F981
:1045800030004FF48041884202DDA8F83010D4E6B4
:104590000028FCDAA8F83040CFE6C749D8F8DC009C
:1045A000884202D2401CC8F8DC0098F80F000828A6
:1045B00003D1D8F8DC0088420ED33470D8F8080054
:1045C000C10502D520F0080001E040F00800C8F85D
:1045D000DC40C8F80800B0E6BDE8F05F02F0D8BCE7
:1045E00098F80F00092804D0A8F8304088F80F4048
:1045F00082E1B24D286A401C2862022809DDA88D9C
:10460000012301B2A88B052200B200F097FA2C62B8
:10461000E862AB48A98D0180B9F844104180FDF7EC
:1046200043FFA8F8300088E6BDE8F05F04F00CBA5C
:10463000A448007809287DD07FE6A048A24984706C
:104640000A8842F480520A8098F8281181B143F315
:104650001101C8F8D8404FEA813C9C4BCAF82C1095
:104660008910C3F828C08A03CAF8281098498A62BA
:104670000483D9F8441041F28830814209DA9AF86B
:104680000010012905D193488AF80040048092481F
:1046900004809249924B0888401C82B291480A805B
:1046A000C82A04D390F800C0BCF1010F1BD0B2F5AA
:1046B0007A7F04D390F800C0BCF1020F13D0B2F59A
:1046C000FA6F02D30278032A0DD098F80F00DFF8B2
:1046D00018B2801E082874D2DFE800F00DADE9E8BA
:1046E0000473749F29E604700C80E88820F400604D
:1046F000E8801F70E9E7FDF70DFE99F800004D46D0
:10470000400611D59BF8020004280DD0686C822861
:104710000ADAA87A95F83D1000F0030001F00301D1
:10472000884201D001F0E4FD3078062884D085F875
:104730003F4000E0E0E0A86C644A40F311008303CE
:10474000CAF82C00801093628103CAF828006048E0
:104750008162FDF7D1FB59484772B8F81401A8F8F7
:104760001601686C4746B0F5437FA8F8824012DD19
:104770004FF48040A7F88000B86840F48060B860CB
:1047800095F838100529ADD140F01000C8F80800A0
:104790008BE03070D1E54FF48041A7F88010B96804
:1047A00021F48061B96040F28A21884204DA2878D5
:1047B000400601D402F0D8FAB86840F01000B860A2
:1047C00073E0B8E0D9F84400B0F5437F07DA9EF80B
:1047D0000010062903D000BF8EF80040A4E0434833
:1047E000017821F040010170FDF786FB43F6FE7071
:1047F000A8F8160108F1DC05FDF78CFD3C4810F81F
:10480000341F21F00101017031492C608C622F4965
:104810008C620821317044648FE52948FDF72CFE35
:10482000FDF76AFB2548D9F84410C16241F27C517A
:10483000C1610920ADE7A879C006ABD4D9F844001E
:104840004D46B0F57A7F57DDFDF764FD28784006C8
:1048500011D59BF8020004280DD0686C82280ADA72
:10486000A87A95F83D1000F0030001F0030188429A
:1048700001D001F03DFD85F83F40B5F84800A8F8AB
:10488000300001B24FF480404446814200DD208672
:10489000FDF732FBA06840F48060A06095F8381006
:1048A0000529B9D140F01000A06023E038E025E0F0
:1048B000B68E000848010020C0D401007802002014
:1048C000AC09002060020020442C0140C8080020F0
:1048D0009808002022000020200000201600002060
:1048E0001400002015000020540400202E07002092
:1048F000700A002002204CE734701EE5D9F844000D
:10490000B0F5437F04DA9EF8001006297FF464AF07
:10491000E88820F02000E880FDF7FCFC042038E760
:104920009EF80000062801D0377006E505490920E9
:10493000087005202DE78BF802408EF800408AF8B9
:104940005E4027E66002002030B585B001210420DA
:10495000FFF79CFA4FF40040ADF8100048208DF8A6
:10496000130004A91848FDF71DFC01210846FFF7B4
:1049700075FA40F68C20ADF8040003240020ADF851
:104980000040ADF80200ADF806004FF080456946E2
:10499000284600F0CBFF1C208DF80C008DF80D4050
:1049A0008DF80E4001208DF80F0003A8FEF752FF8E
:1049B00001221146284600F093FE0121284600F00E
:1049C000C1FD05B030BD0000000801407047000087
:1049D0002DE9F041304CE07800285AD120780028A9
:1049E00057D0401E10F0FF00207052D14FF4967047
:1049F000208272B6294F45F2AA50A7F87200002013
:104A0000FDF758FA264D13202860FDF765FAA8BB7C
:104A10003420E86002202861224E6E61286940F04F
:104A200040002861FDF758FA40BB00211E4A0846A5
:104A30005FEA255312F800C0BCF1FF0F00D001213E
:104A4000401C80B29842F5D3C1B9C4E90676392634
:104A50000127A06910F8011B10F8012BA061E06983
:104A600001EB022102886A612F6120F8021BE061DC
:104A7000FDF732FA10B9761EB6B2EAD20120FDF780
:104A800019FA62B601F088FC0848816821F4804177
:104A90008160BDE8F08100001C070020BC0C0020F4
:104AA0000020024000FC000800FC0008A8020020D2
:104AB0001948016841F010010160016821F003010B
:104AC0000160016841F002010160144841684160E1
:104AD00041684160416841F480614160416821F46E
:104AE0007C11416041680E4A11434160016841F008
:104AF0008071016001688901FCD5416821F00301E2
:104B00004160416841F0020141604168C1F38101A7
:104B10000229FAD170470000002002400010024034
:104B20000000280830B5044C039D6080A180E2801D
:104B30002381658130BD0000500A00200A44824272
:104B400001DA10B27047C91A8142FBDD08B2704722
:104B50002DE9F0434348DFF81081DFF81091C17F61
:104B6000457A046801260023414A424880292BD314
:104B700001F01F0158F821100C420146096802D0CB
:104B800041F4805101E021F480510160CF0417D439
:104B90008F0415D5977AFF0707D0538199F800C085
:104BA0002CF0020C89F800C00AE090F84670BFB102
:104BB0004FF0020C012F18D080F8463080F81AC14F
:104BC0000F0B67F34D310160802D2AD305F01F01D3
:104BD00058F821100C4201680CD041F004010BE0A0
:104BE00080F8466080F81A31EAE780F846C080F81D
:104BF0001A61E5E721F0040101604C070DD44C0572
:104C00000BD5947AE40708D0538199F8005025F029
:104C1000020589F80050C0F898308C0864F38A21A6
:104C20000160917AC90717D1134991F864100129DD
:104C300012D11249496C32290CDC0178490709D597
:104C40000189090506D4D0F8981047F23054A142E2
:104C500004D95681C0F89830BDE8F083491CC0F8EB
:104C60009810F9E7E40500208C940008DE05002088
:104C70005C0A0020A8020020BC0C00204801002093
:104C800010B5FCF76FF80F48018821F00201018090
:104C90000C49183109880C4A928E1144094A343261
:104CA000118008490C390A8842F001020A80011D6E
:104CB0000A884FF6ED531A400A80018841F012012C
:104CC000018010BD0C0400405404002006484188B7
:104CD000491C89B24180B1F57A7F04D38188491C8F
:104CE0008180002141807047400700200F4810B5A7
:104CF000016841F00101016041680D4A11404160C5
:104D000001680C4A11400160016821F480210160B2
:104D1000416821F4FE0141604FF41F018160FFF7FB
:104D2000C7FE05494FF00060086010BD001002404A
:104D30000000FFF8FFFFF6FE08ED00E02DE9F0416E
:104D40003149324D0888401C088028884FF0000403
:104D5000000629D5FCF786F92D4A2E480723177837
:104D6000C8262D49012F22D02C4FB7F806C0BCF120
:104D7000000F3ED0B0F80CC04CF0080CA0F80CC0EE
:104D8000B0F806C02CF4006CA0F806C0886820F0CB
:104D900004008860FC801370CE8700204FF4966179
:104DA000401C80B28842FBD32C80BDE8F0811C4FB0
:104DB00097F800C0BCF1010F0FD0BCF1020F11D069
:104DC000B0F806C04CF4006CA0F806C0886840F04B
:104DD0000400886005203870DDE7B0F80CC04CF0A6
:104DE000080C03E0B0F80CC04CF0100CA0F80CC09C
:104DF000F0E70C4F3C70C78847F40067C7808868AD
:104E000040F004008860C6E740070020102C0140F5
:104E10001F0700205C0A0020A8020020680900206B
:104E2000200700203D070020704700002DE9F043D7
:104E30004FF08040018A21F001010182AC480078E6
:104E400000287CD1AB4FF87B002878D1AA48406C71
:104E5000322874DCA9488068DFF8A4924104A94D87
:104E6000B9F804004FF0000403D4401CA9F8040072
:104E700028E1002874D02978012611B1012912D027
:104E800017E14946B0F5BE7FFAD92E70CC718C710E
:104E9000EC702C72287A0A18401CC0B21472287266
:104EA0000F28F7D305E1B9F802204946824201D91B
:104EB000EE7100E0EC7192488A7908300F2A15D221
:104EC000CB79082B0BD2C3F10708EB7912F800C09D
:104ED00003FA08F363441354CA79521CCA71CA799D
:104EE000082A03D18A79521C8A71CC7199F806106C
:104EF000C8460F2973D10D21FCF71EF8A881010ABD
:104F00006970C0B2A87088F8064098F816208A42E6
:104F100065D198F81510814261D198F80BC07A4993
:104F2000032302227948BCF1000F10D0BCF1010F1D
:104F300002D0BCF1020F14D080F86A2000E0CBE070
:104F400091F800C02CF00C0C0CF1080C0FE080F86C
:104F50006A6091F800C02CF00C0C0CF1040C06E017
:104F6000A9E080F86A3091F800C04CF00C0C81F890
:104F700000C098F80C10B6EB111F04D180F86E40F9
:104F800087F846400EE0B2EB111F04D180F86E6046
:104F900087F8466006E0B3EB111F03D180F86E205E
:104FA00087F846200B0717D001F00F01012901D027
:104FB000022915D080F86C602C7198F80D102A79B0
:104FC00006FA02F30B406B71082A44D2DFE802F0C4
:104FD0000B124319242F363D80F86C40ECE768E053
:104FE00080F86C20E8E713B180F8704033E080F877
:104FF000706030E013B180F850602CE080F85040D1
:1050000029E023B180F8656087F8036123E080F828
:10501000654087F803411EE023B187F8F54080F82A
:105020004D4018E087F8F56080F84D6013E013B14B
:1050300080F868600FE080F868400CE013B180F8F9
:10504000666008E080F8664005E013B180F86760AC
:1050500001E080F86740521CD2B22A71082AAED310
:1050600098F80E102A4A8B0705D587F8F16080F86A
:105070006460568104E087F8F14080F86440548110
:10508000C90702D080F8294001E080F8296098F82B
:10509000111000F86D1FC2781E48012A1ED001B3FE
:1050A000012921D04FF48051A0F876101A493C20F4
:1050B0000870A9F80240A9F80440B9F80210491C88
:1050C000A9F80210B9F80210B1F5FA7F04D940F23C
:1050D000F511A9F802102C70BDE8F08344F21C71A0
:1050E000E2E74FF40051DFE741F25551DCE7000001
:1050F0001F070020A80200204801002000100140E6
:10510000A40C0020B8060020CC040020BC0C002019
:105110005C0A0020340500201C0700202DE9F05F08
:10512000FDF7F8F88E4D2888A5F10406C0070AD0CF
:10513000308820F008003080288820F0090028807E
:1051400001F012FED9E02888DFF81892DFF8188203
:10515000864C80071AD5B9F8001041F00101A9F872
:105160000010B8F8000080491431503008802888B9
:105170004FF6F95108402880308840F00400308014
:10518000FEF7F0FE84F83C00BDE8F09F2888784FD9
:105190004007288871D520F004002880FEF7E2FE41
:1051A00094F83C108142EFD1308820F00400308028
:1051B000FDF788FA2078410605D594F84C1094F84C
:1051C0003B209142E0D03978400621F0020139704D
:1051D00004D5FEF7A3F997F82F7004E094F83C008B
:1051E000FDF7EAF80746DFF880B140F68C2A0BF1AC
:1051F000180B062F47D294F83800B8423ED03846F4
:10520000FDF75EF82078C00716D094F83A0094F8BD
:10521000391000F00302914206D0A17A00F001009B
:1052200001F00101884215D1FDF7B4F9FBF7E6FD65
:10523000FDF7DCFA384689E0FDF7ACF9FBF7DEFD57
:10524000FDF7D4FA3846FDF7C5F9207840F00100A3
:10525000207099E7288820F008002880206B8108BA
:1052600001EBD000504515D2B8F800100844ABF857
:105270000000308840F0080003E00DE0308820F0A6
:105280000800308080E7B9F8001041F00101A9F86A
:105290000010DFE75046E7E70007288831D520F007
:1052A00008002880308820F008003080FEF75AFE81
:1052B00084F83C00FDF706FA387820F002003870D8
:1052C0002078400604D5FEF729F997F82F5004E01E
:1052D00094F83C00FDF770F80546062D08D294F8C6
:1052E0003800A842B5D0FDF755F9FBF787FD2AE055
:1052F0002048C18841F04001C180BDE8F05FFDF762
:1053000055BAC006288825D520F01000288030889E
:1053100020F01000308097F838000C2802D2401C92
:1053200087F83800387840F002003870FEF7F6F859
:1053300097F82F50787884F8390094F83800A8420C
:1053400087D0FDF727F9FDF751FA2846BDE8F05F51
:10535000FDF740B94EF2BE110840288014E7000066
:1053600010040040000400402404004048010020D4
:10537000540400205C0A00202DE9F04F514F85B005
:10538000388820F0010038804E4800261030068012
:105390004D4CDFF838A14FF0010894F85C0042F65C
:1053A0003029C10774D072B64948816941F400714F
:1053B0008161816941F4806181614FF40040FEF7B1
:1053C00037FD444D00212846FBF776FA0021284698
:1053D000FBF768FADFF800B100215846FBF762FAE4
:1053E00000213E48FCF7E2F82846FBF781FB5846CF
:1053F000FBF77EFB4FF46020CDE902068DF80560D7
:1054000000968DF810808DF8048069462846FBF7D9
:1054100001FC01231A460F212846FBF74CFC012111
:105420002846FBF73FFA00204946401C80B28842DC
:10543000FBD328462E600121FBF77CFC28688007FF
:10544000FCD524484C30006894F85C1021F0010130
:105450002144A1F85000FBF739FA62B6FDF76AFF64
:1054600047F69061AAF8001094F85C00401CC0B2A6
:1054700084F85C000C2822D212491431A1F8008073
:10548000388840F00100388005B0BDE8F08FFFE7B4
:10549000134920F00100085A12490880114945F6C5
:1054A0005800083908800F4847F25801001F018052
:1054B0000C4920200C390880AAF80090D4E703207A
:1054C000A070E1E700080040540400202C080040D0
:1054D0000010024000240140002801400800024062
:1054E00048900008202C01400029018802D041F09A
:1054F000800101E021F080010180704710B50A8829
:105500004B88CC881A438B8823431A430B891A4350
:105510004B8989891A430A43A0F8442010BD002111
:10552000018041808180C1800181418181817047FA
:105530000029818802D041F0010101E021F0010140
:10554000818070470029018802D041F0010101E00B
:1055500021F0010101807047002930F8441F02D07A
:1055600041F4004101E0C1F30E01018070470000E9
:105570004B4910B5884202D10121C41486E0B0F134
:10558000804F09D0474988420DD101210220FEF702
:1055900071FC0021022064E001210846FEF76AFC4C
:1055A000002101205DE04049884206D1012104200C
:1055B000FEF760FC0021042053E03C49884206D1FC
:1055C00001210820FEF756FC0021082049E0384957
:1055D000884206D101211020FEF74CFC002110204A
:1055E0003FE03449884206D101212020FEF742FCE9
:1055F0000021202035E03049884202D101214414A5
:1056000044E02E49884202D10121CC043EE02C49DD
:10561000884202D101210C0538E02A49884202D192
:1056200001214C0532E02849884206D10121402061
:10563000FEF720FC0021402013E02449884206D1D7
:1056400001218020FEF716FC0021802009E020497E
:1056500088420AD1841501212046FEF70BFC002167
:105660002046BDE81040FEF705BC1A49884202D129
:1056700001210C040AE01849884202D101214C049E
:1056800004E0164988420AD101218C042046FEF725
:1056900009FC2046BDE810400021FEF703BC10BD08
:1056A000002C01400004004000080040000C0040B5
:1056B000001000400014004000340140004C014044
:1056C000005001400054014000180040001C004000
:1056D00000200040004001400044014000480140DB
:1056E000002A828901D00A4300E08A438281704700
:1056F00030B5028C22F001020284028C8388048B74
:1057000022F0020224F073050C882C430D89154306
:105710004A882A43114DA8420BD0114DA84208D007
:10572000104DA84205D0104DA84202D00F4DA842FE
:105730000DD122F008054A8923F440732A4322F050
:1057400004058A882A438D891D43CB892B43838096
:105750000483C9888186028430BD0000002C01408A
:105760000034014000400140004401400048014035
:10577000028B22F008020A430283704770B5028C44
:1057800022F010020284028C8488038B0D8823F49B
:10579000E6464FF6FF7303EA052535430E8922F0EE
:1057A000200203EA061616434A8803EA021232432D
:1057B000104EB04202D0104EB04215D122F08006F9
:1057C0004A8924F4406403EA0212324322F040067C
:1057D0008A8803EA021232438E8903EA8606264348
:1057E000CC8903EA8404344384800583C988018713
:1057F000028470BD002C014000340140028B4FF642
:10580000FF7322F4006203EA012111430183704710
:1058100070B5028C22F480720284028C8488838B9F
:105820000D8823F073031D4322F400730E894FF695
:10583000FF7202EA06261E434B8802EA0323334323
:10584000104EB04202D0104EB04215D123F4006683
:105850004B8924F4405402EA0323334323F4806643
:105860008B8802EA032333438E8902EA0616264315
:10587000CC8902EA0414344384808583C9888187F3
:10588000038470BD002C014000340140828B22F063
:1058900008020A438283704770B5028C22F480525A
:1058A0000284048C8288838B0D8823F4E6464FF6AD
:1058B000FF7303EA0525354324F400560C8903EAF7
:1058C000043434434E8803EA06362643094CA0428A
:1058D00002D0094CA04205D122F480448A8903EA0F
:1058E0008212224382808583C988A0F840100684F2
:1058F00070BD0000002C014000340140828B4FF647
:10590000FF7322F4006203EA01211143818370478F
:10591000018582827047828822F0700282808288AC
:105920000A4382807047A0F84010704730B5028863
:105930001B4B1C4C98420DD0A0420BD0B0F1804FB5
:1059400008D0194DA84205D0184DA84202D0184DD4
:10595000A84203D122F070054A882A43154DA84277
:1059600006D0154DA84203D022F44075CA882A43B8
:1059700002808A8882850A88028598420AD0A042DD
:1059800008D00E4A904205D00D4A904202D00D4AEE
:10599000904201D1097A01860121818230BD000047
:1059A000002C014000340140000400400008004089
:1059B000000C004000100040001400400040014076
:1059C00000440140004801404FF6FF7181800021F2
:1059D0000180C1804180017270470029018802D096
:1059E00041F0020101E021F002010180704700292D
:1059F000018802D041F0040101E021F0040101809E
:105A000070470000224910B591F820000A6821492A
:105A100000F01F0051F820001F490242086802D020
:105A200040F4803001E020F4803008601B484FF0E3
:105A30000003807941061A4827D41A4902880C8845
:105A4000A21A92B201240F2A0BD30A88028082681C
:105A5000002A00DA5242062A03DD134A1278022A8B
:105A600005D0427F012A06D00988418010BD4477C5
:105A7000C3770A88428042880988891A89B240F22D
:105A80001A629142F2D3C47710BD437710BD000073
:105A9000E40500208C940008A80200205C0A002085
:105AA000840C0020280700201F0700202DE9F0416A
:105AB0004D6800231E240F22854202DD0868BDE8E0
:105AC000F081D1F8F450854202DAD1F8F000F6E71F
:105AD00001EBC2056D68854201DA134600E0144609
:105AE000E21852085D1CAA42F2D101EBC20351F840
:105AF00032505C68844202DAD3E9026701E053E97C
:105B00000267001BC11789053A1B41EA9021D31790
:105B10008005FAF707FB721BA0FB024601FB02613E
:105B2000D31700FB0310810241EA94502844C6E7D2
:105B30002DE9F04FDFF8B8B16A48DFF8AC91DFF833
:105B4000ACA190F80EC0BBF91A70BBF91C60BBF990
:105B50001850BBF96C10BCF1070F48D2DFE80CF00D
:105B60008D041A30485E7600D9F800208284DAF875
:105B70000020C284828CC38CA7EB820212B2A6EBF7
:105B800083034A431BB2594342F3CF2241F3CF234D
:105B9000D11870E0D9F800204284DAF80020C284DD
:105BA000428CA5EB820213B2C28C4B43A6EB82025D
:105BB00012B243F3CF24514341F3CF23E11814E051
:105BC000D9F80020C284DAF800204284C28C438CC9
:105BD000A6EB820212B2A5EB83031CB24A436143D7
:105BE00042F3CF2341F3CF24191949420AB244E0CA
:105BF000D9F800208284DAF800204284828C438C19
:105C0000A7EB820212B2A5EB83034A431BB25943AE
:105C100042F3CF2241F3CF24111914E0D9F8002028
:105C20004284DAF800208284428C838CA5EB8202C5
:105C300012B2A7EB83034A431BB242F3CF2459436A
:105C400041F3CF22A11849420BB216E0D9F8002047
:105C5000C284DAF800208284C28C838CA6EB820294
:105C600012B2A7EB83031CB24A4342F3CF23614332
:105C700041F3CF22991849420CB2BBF91E50594644
:105C800005F21E56A64201DACE8306E0A5F21E55A5
:105C9000A54201DDCD8300E0CC83B1F9204004F2C0
:105CA0001E55954201DA0D8406E0A4F21E5494427A
:105CB00001DD0C8400E00A84B1F9222002F21E54B6
:105CC0009C4202DAABF8224008E0A2F21E529A424D
:105CD00002DDABF8222001E0ABF82230417B81737A
:105CE000BDE8F08FA80200203C2401403C28014080
:105CF000340500202DE9F04704466F48704D00261A
:105D000002786E48022AB0F9301004D0082A7BD0FD
:105D1000092A7AD0CBE0C27B022A02D1B0F8402017
:105D200052B1A4F8421069810423B5F908101A464B
:105D30000020FEF703FFB1E06249DFF88C81496A79
:105D40000F14E7808068410216D5B4F9020040F2D2
:105D5000DA21884248DD40F26A41884205DD00BF11
:105D60000823B4F942101A4660E0A0F2DA20FAF7EC
:105D700054FB0022554B68E0C0F3C001C0F3002083
:105D8000DFF84C9181420CD1D8F8440040F2BA417E
:105D900088426DDD40F66A118842E1DCA0F2BA402B
:105DA0004FE04C480078C0060CD5D8F8440041F2CA
:105DB000243188425CDD41F2D4718842D0DC00F6A7
:105DC000DC401EE04448DFF8149190F8701001297F
:105DD0000BD090F86F00012807D041480178C9071F
:105DE00046D04049098889B142E0B4F9020041F641
:105DF000DC6188423CDD42F23411884212DC00F55D
:105E00009270A0F500501CE04AE04EE0B0F910009E
:105E1000B4F90210A0F59672914229DD00F5967250
:105E200091420BDDB4F9421020231A460020FEF700
:105E300085FEA4F84200002817DB1BE0081A00F5D5
:105E40009670FAF7EAFA00224B46FAF752FA0E2257
:105E5000FAF7BEFAFAF718FB00B2C0F580407843B3
:105E60008013A4F84200002F04DCA4F8426001E093
:105E7000A4F84270B4F842001B4FE880D8F84410F0
:105E80007964A7F84C0000F083FBB7F84E006881F6
:105E900098F80A000028388F00D14042288106E097
:105EA0001248B0F87C00688100E069812E8184F896
:105EB0004060BDE8F08700001F070020A802002016
:105EC00064000020340500204801002000007940D3
:105ED00000C0924000070020BC0C002000C082409F
:105EE0004C09002020000020F8080020700A002043
:105EF0002DE9F041B1F9025000232B2415228542EF
:105F000003DAB1F90000BDE8F081B1F9AE50854285
:105F100002DDB1F9AC00F6E701EB8205B5F90250FC
:105F2000854201DD134600E01446E21852085D1C6C
:105F3000AA42F1D101EB8205B5F90230834206DABB
:105F400035F9026C35F9044C31F9221006E01E4691
:105F500031F92240B5F90630B5F90410801B091B50
:105F6000C5178911AD0345EA90458703A1FB070CCE
:105F7000CA1702FB07C201FB05219A1BD317FAF7C8
:105F8000D1F8000A40EA0160001900B2B0F5804F74
:105F9000B9DB43F6FF70B6E770B5134C40F2244509
:105FA0002946204600F03EF800281BD0204600F08D
:105FB000C7F82946204600F01DF80C4C0021204669
:105FC000FBF7F4FA2046FBF76FFBC0F164000849C9
:105FD000C0B20428087201D900F046F9BDE870404B
:105FE000FBF7A8BB70BD000000380140580002401C
:105FF000700600200A0A01219140C94301807047C0
:106000000029818902D041F4005101E021F40051BE
:1060100081817047002A828A01D00A4300E08A43C6
:106020008282704730B501F01F0201240025C1F3C0
:10603000421304FA02F2012B0FD0022B0FD0838AF5
:106040004FEA11210088134204FA01F400EA040027
:1060500001D000B10125284630BD8389F0E7038ACD
:10606000EEE710B5C1F3421301F01F040121A14076
:10607000012B07D0022B07D01430002A026805D06C
:106080000A4304E00C30F8E71030F6E78A43026078
:1060900010BD000030B50446008A85B00D464CF6B0
:1060A000FF710840E98801432182A1894EF6F3106F
:1060B0000140A8882A8910436A890A431043A081B5
:1060C000A08A4FF6FF410840A9890143A182684692
:1060D000FDF7F4FE1948844201D1039800E00298CC
:1060E000A189090400EBC00101EB0010296801D56A
:1060F000490000E08900B0FBF1F06422B0FBF2F14E
:1061000009010B096FF018056B4300EB8300A389AD
:106110001D044FF0320306D503EBC000B0FBF2F0D4
:1061200000F0070005E003EB0010B0FBF2F000F018
:106130000F000843208105B030BD00000038014049
:106140008088C0F308007047F8B501210920FDF7E9
:106150009DFE01218803FDF799FE10258DF803505F
:106160002020ADF800001A4E03248DF80240694645
:106170003046FCF717F816490C31086820F020006B
:10618000086018208DF803004020ADF800008DF85D
:10619000024069463046FCF705F848208DF80300B8
:1061A0008020ADF8000069463046FBF7FBFF8DF814
:1061B00003502801ADF800008DF8024069463046D2
:1061C000FBF7F0FF01210420FCF73EF8F8BD0000CA
:1061D000000C014030B585B0FFF7B6FF00244FF446
:1061E000E1300090ADF808400C201D4DADF80440A2
:1061F000ADF80A00ADF80640ADF80C4069462846F7
:10620000FFF748FF25208DF8100004208DF81100BD
:106210008DF8124001208DF8130004A8FDF71AFB39
:10622000012240F224412846FFF71BFF01212846A6
:10623000FFF7E6FEFBF7A8FA012280212846FFF7C8
:10624000E9FE012240212846FFF7E4FE0122022157
:106250000448FBF73DFAFBF797FA05B030BD0000A4
:10626000003801404400024070B51D4D00242878DC
:10627000432834D16878462831D1A878502807D0EF
:10628000512805D0812803D0892801D0212826D182
:10629000144E7071E9787172A81C891CFAF784FE9B
:1062A000B072717A294409793182884217D106F196
:1062B0000E00017841F0020101700B48016841F0C5
:1062C00020010160317A0948002204E02B5D03556A
:1062D0002A55641CE4B28C42F8D38078707170BD8A
:1062E000B8070020700600200C0C0140EE0B0020C7
:1062F00070B51D20FDF78DFAFDF710F91D20FDF793
:106300009EFA154890F82F10144D0623144C85F86A
:10631000381090F83B1095F83B201143012A04D027
:10632000022A07D0042A0AD010E0827A8A420DD0CD
:10633000007B09E0027D8A4208D0807D04E0827FF4
:106340008A4203D090F82000884200D123700020B8
:1063500085F8400070BD0000540400204801002072
:106360001F0700200B4800214180A0F1B0018A895D
:106370008280CB891A44C2800B8A1A4402814B8ADC
:106380001A444281898A1144818143F6FF71C18197
:1063900070470000F8010020084940F61C72B1F96E
:1063A0000C00904202DA00F59F7005E041F2E30232
:1063B000904201DDA0F59F70C88170476400002005
:1063C00038B51348C16941F00401C1611E208DF840
:1063D000000002208DF801008DF8020001248DF8E4
:1063E00003406846FDF736FA0A49842008800949C7
:1063F00047F690602C3108800020091F088005496D
:1064000014310C80091F0880081F048038BD00006B
:10641000001002400008004030B420491E4A457870
:106420008B7A114692F83B4091F83910AC4218D162
:106430004BB10379994202D04379994201D1407915
:106440001AE0807909E08379994202D0C479A142A7
:1064500002D182F82F3011E0407982F82F0030BC51
:106460007047C578AC42FAD16BB1C379994202D07A
:10647000037A994205D1007A82F82F0030BCFEF7EA
:10648000FFBB407AE9E7437A9942E2D00479A1421E
:10649000DFD0007AE1E7000054040020480100202A
:1064A000FEE700002DE9F0470446007F012868D18F
:1064B0003548E1880288511A89B2072916D3008825
:1064C000E080B4F9000044F2DD414843401346F651
:1064D000D96148438013A060401000B2A0814FF002
:1064E0008051B1FBF0F0F9F793FF2061B4F90C6033
:1064F00096B1B4F902104DF6B05048430014A08292
:10650000B4F904704DF6B05207FB02F24FEA22458F
:10651000E58204D4024603E00020E08330E04242FA
:1065200012B22283002D01DB2B4600E06B421BB22E
:10653000DFF85890638398464FF4804AB24208DAF5
:10654000F9F75DFF2169F9F730FEF9F784FF801351
:1065500004E0002901DA484600E05046E083B045F7
:1065600009DA2846F9F74BFF2169F9F71EFEF9F71A
:1065700072FF801304E0002F01DA484600E0504625
:106580002084BDE8F08700002807002000C0FFFF3E
:1065900010B52248234C01782148022905D1C17B3E
:1065A000022902D1B0F8401029B1008EA4F84E00A3
:1065B0000020208710BD90F846101A48B0F844001B
:1065C00000B239B318490978C1F3810101291BD000
:1065D00002291CD0154900BFFBF73CFC1149A4F867
:1065E000400080B2483101F091FAB4F94C00B4F99E
:1065F0004A2041425143891324F8381FB4F910103E
:1066000048438013E08210BD0849D839E4E70749C0
:106610006C39E1E705496C31DEE700001F07002017
:10662000A8020020F8080020CC040020C08D00083B
:106630000348002180F82A10C183018770470000B9
:10664000F808002010B504000B462D4AC3F10000E5
:1066500028D56442002B12DAA04207DA214600F066
:106660002DFA32F81000C0F5404041E001462046C6
:1066700000F024FA32F8100000F5004038E0A342A0
:1066800008DA2146184600F019FA32F8100000F531
:1066900040402DE0204600F011FA32F81000C0F51D
:1066A000803025E0002B12DAA04207DA214600F004
:1066B00005FA32F8100000F5804019E00146204646
:1066C00000F0FCF932F81000C0F5004010E0A342E1
:1066D00008DA2146184600F0F1F932F81000C0F54A
:1066E000804005E053B1204600F0E8F932F8100090
:1066F000B0F5004F01DDA0F5803010BD002010BDC9
:106700005490000840438013494300EBA13000221D
:106710000302002B14DDB3F5001F01DC802001E033
:106720004FF4005093FBF0F1014401EBD17149109B
:10673000814206D0521CD2B20846062AF2D300E0AB
:106740000021C80000B2704702E008C8121F08C14B
:10675000002AFAD170477047002001E001C1121FE2
:10676000002AFBD1704700002DE9F047A74CA8484C
:1067700021880288511A89B20F297DD30088A4F19B
:106780003C052080288F08B1401E288795F800C05E
:10679000A04ACCF3810001281DD0022820D0D18B43
:1067A0009D4E9A48DFF87492F388407E0027B1F539
:1067B000926F1CD8142818D37820607643F010000C
:1067C000F08040F26660A8812CF001002870D77339
:1067D00089F8007018E0D08B00EB4000C00302E0A5
:1067E000D08B8F494843010CDAE7401C04E0B1F537
:1067F000DB6F09D310B1401E607605E023F0100076
:10680000F0804CF001002870B5F90200B5F91430A1
:106810004143C3EBC303C1F38F31C3F3D10303EB94
:10682000510109B2A9829046D28B4FF08053504358
:10683000B5F91620C0F38F30C2EBC202C2F3D10209
:1068400002EB500000B2E882AA6A42431213EA62E5
:1068500093FBF2F22A63734A1080A2680A44A26092
:10686000E1680144E160207C401CC0B2207407282C
:1068700002D942F3CF0000E0C5E02883C910698344
:10688000E760A76041F6C8012774884204DD298BC0
:10689000654AB2FBF1F1E981C117890341EA9041F0
:1068A000800342F69B420023F9F73CFCA88457483A
:1068B0005E49A0F13C002A78B0F906005FEA827CCC
:1068C00000FB01F14FEA2143C2F3810115D50129F3
:1068D00007D002290BD04FF2685141430914A1801F
:1068E00011E049F68C4148430014A08020E04CF6AA
:1068F000183141430914A18026E001290ED0022954
:1069000018D0A0806B844A4948430014A4F81E00A4
:10691000FBF7C0F847480088C0B143E04AF65C3155
:1069200041430914A1804BF62C214843001468848C
:10693000E383EDE74DF2AC5141430914A1804EF2DF
:106940007C414143091469843B49DDE795F8200007
:1069500000BB88F80F7089F80070B5F91A00A0F52F
:106960000C519F39B1F56E7F18D8617FF42912D987
:106970003249E8802E4AA1F8460050430014A8800E
:10698000A1F84400FF2085F8200081F828002C4958
:106990003C20087006E0491C617703E0607F08B185
:1069A000401E6077B5F91A10B4F91E0081420EDD61
:1069B000A07E7D2809D9F08840F00800F0802148A9
:1069C000017821F0020101700EE0401C06E0A0F207
:1069D0003D10814208DAA07E10B1401EA07603E08F
:1069E000F08820F00800F080B5F9181060690844BC
:1069F0006061217E491CC9B221761F2903D940114B
:106A0000A88367612776BDE8F087000008050020AD
:106A100028070020A80200205C0A00201F07002091
:106A200030330100100A002074E8260BCC0E010060
:106A3000488501002A070020D0450100BC0C002039
:106A40001C070020DE050020024941F68B308862D9
:106A500070470000CC04002070B5164C0625207845
:106A6000062825D2DFE800F003080E141A21124888
:106A7000FAF7D8FA012016E00F48801DFAF7D2FA8B
:106A8000022010E00C480C30FAF7CCFA03200AE0A0
:106A900009481230FAF7C6FA042004E00648183014
:106AA000FAF7C0FA0520207070BDFAF7DBFA2570FE
:106AB000257070BD20070020988E0008090A05D0B7
:106AC000B0FBF1F0FF2800D9FF207047002070478D
:106AD000D0E90021C368521A5A4301EBA231816008
:106AE00041607047B0F90020B0F90210B0F90630EB
:106AF000521A5A4301EBA231818041807047000055
:106B000030B5494B188849490A8A801A85B24848E5
:106B1000484A0F2D047801F150001DD31D880D82C5
:106B2000117A090713D5022C01D0434912E0434DD5
:106B3000B0F90210B5F90050A94205DC02DA01F102
:106B4000020108E0458007E0A1F1020103E0022C08
:106B500002D13B4909884180B0F840101D88691A6C
:106B600089B29C2949D31988A0F84010916A002362
:106B7000B1F5804F31DB3349896CB1F5405F2CDDD5
:106B8000314940F26665B1F91010A94212DD43F6B1
:106B90009915A94202DB40F2333108E040F2333567
:106BA000A1F26661694343F2333591FBF5F1A0F838
:106BB000441001E0A0F844302449B2F806510978A5
:106BC000C1F381012DB100BFB0F8441001F21E5194
:106BD0001CE092F84620022A10D0A0F84430022C83
:106BE00001D0A0F84430B0F95C10B0F9443001F1A4
:106BF00014029A420DDAA0F85C2030BD012901D0C0
:106C00000229E1D1B0F8441001F23331A0F8441068
:106C1000E5E703F11402914203DD1439A0F85C109A
:106C200030BDA0F85C3030BD2807002014000020E3
:106C30001F070020A8020020CA040020C80400206A
:106C4000C40400204801002034050020CC040020AA
:106C50002DE9FC4101210220FDF700F90121192055
:106C6000FDF714F901213C48FBF7EEFA4027ADF897
:106C7000007003248DF802400420384D8DF8030085
:106C800069462846FBF78EFAE001ADF800008DF862
:106C900002401C208DF8030069462846FBF782FA63
:106CA0004FF4E0712846FBF704FBA815ADF800008F
:106CB0008DF8024010208DF8030069462848FBF744
:106CC00071FA4FF4A060FCF7F7FD1D208DF8040069
:106CD00001268DF8056000258DF806508DF80760B7
:106CE00001A8FCF7B7FD1F498C2008801D494FF60D
:106CF000FA702C3108806E20091F08801948143062
:106D00000680184808300780164920310D80154A42
:106D1000D020121D1080134A45F2F3001832108063
:106D20000A1F45F2500010800E4A4FF6FF703832AD
:106D30001080121D1080121D108041F21B1008805F
:106D400000F012F8FBF732FD064810300580001FF6
:106D50000480BDE8FC810000000C1A000010014016
:106D6000000C01400004004070B51D20FCF746FDFA
:106D70002A4D40212846FBF793FA840080212846BB
:106D8000FBF78EFA44EA4004A9152846FBF788FA77
:106D90000443E0B2224C84F83C00FBF70DFB0546AF
:106DA000052805D91F48C18841F04001C18001E094
:106DB00084F838501C48007A000703D594F838004E
:106DC0001A490D5C4FF6FA702063E062A0626062BF
:106DD0002062E061A0611648606300206064A064E6
:106DE00084F83F0084F84000FBF794FAA07AFF286B
:106DF00011D0022084F83D000E4800882066284605
:106E0000FBF736FF207820F001002070BDE87040CD
:106E10001D20FCF709BD0120ECE700000010014037
:106E2000480100205C0A0020A802002050990008B8
:106E3000DCFF0500240400402DE9F0434E484F4993
:106E400002880B889A1A92B20F2A69D309880180A6
:106E50004B49098B027D00EB42029180017D491C68
:106E6000C9B2017508295BD3002404752246017D4F
:106E700000EB4103491CB3F90430C9B202EB6302D1
:106E800012B201750829F2D33E4904753E4B4A807F
:106E900044800E789D895FEAC67C40F638694FF0E1
:106EA000030714D0A2F22B5C42F6E858C44520D365
:106EB000A1F1020C26F00204ACF8002047750C701A
:106EC00040F22B54A24211DA45F004021EE046F0D3
:106ED00001060E704A4507DD45F001029A8126F051
:106EE00002020A70477519E0447517E045F0020286
:106EF0000CE04A450CDA8775427D12B1521E42758C
:106F00000CE046F002020A7025F007029A8105E0C3
:106F1000B30703D5837D2BB15B1E837540888880C2
:106F2000BDE8F08342F6AA239A4222DAB1F904308E
:106F30002BB941F2CD05AA4201DA4480EEE7134CA9
:106F4000920302EB843241F67244B2FBF4F214B2C3
:106F500040F2333502464480AC4200DA5580B2F943
:106F60000240E41A04F5A374B4F5237FD6D8438015
:106F7000D4E74FF48043FAE7F00A00202807002006
:106F8000A8020020DE0500205C0A0020C8F1FFFFF7
:106F90002DE9F0416D4CDFF8B8E14FF0000594F8B1
:106FA0003410C80706D094F938104B42002958DD38
:106FB0000E4657E0674884F83750A4F84250664AB6
:106FC00090F8380084F840001586CEF80450CEF8CA
:106FD0000850624E40F26663CEF80C50A4F87C3044
:106FE00036F810005E4E768830444FF6FF7606EA9B
:106FF000800024F8300B4FF0806044F8040CA3208C
:10700000208460845810A084E38440F69910208581
:10701000580060854FF48050A08541F23330E08500
:1070200041F26660208641F69910608641F6CC40B8
:10703000A0864FF40050E08642F23330208742F2BF
:107040006660608742F69910A08742F6CC40E087E0
:1070500082F89D5041F00100207184F84450BDE851
:10706000F0811E4694F937004242002801DD0746B0
:1070700000E01746F61B012E0BD0002800DB02466D
:107080005FFA82F684F8380094F84F00012805D0A2
:1070900041E0002900DA1946CEB2F3E794F939301D
:1070A0005942002B01DB184600E0084694F93A20CB
:1070B000C7B25042002A01DB944600E08446BC453A
:1070C00008DD002A00DA0246D7B2002B00DA0B46B0
:1070D000D8B207E0002B00DA0B46DFB2002A00DB53
:1070E0001046C0B204EB4000B0F9501004EB47006A
:1070F00030F9502F11444910018084F84F5084F822
:107100003E5084F83D5084F83C5084F83B5084F85D
:107110003A5084F8395004EB46007546B0F95000F7
:1071200024F8420FBEF80410C82309B26422FDF708
:1071300005FD6860E968401AA9680844A860B5F9C7
:1071400000104843C013E860608788E7700A002099
:10715000CC05002048010020A80200206299000808
:1071600064000020F0B4544890F83410C90776D079
:10717000524990F84030002291F838108B426FD07D
:107180004F4CA0F872204F4DE65C04468E4294F9B5
:10719000374002D0EE5C8E420FD1641C64B280F89E
:1071A0003740EB5C8B4202D1641C80F8374090F989
:1071B00037300F2B1BDD0F2317E0434DEE5C434DA3
:1071C0008E4202D0EE5C8E4211D1641E64B280F811
:1071D0003740EB5C8B4202D1641E80F8374090F957
:1071E00037406FF00E039C4201DA80F83730324BA3
:1071F00090F83F50393390F83740EC5490F83F30D6
:107200005B1CDBB280F83F30062B01D380F83F20B7
:1072100090F9394090F93B309C420ED190F93D40B5
:10722000A3420AD190F93A4090F93C309C4204D1F3
:1072300090F93E40A34200D1012280F84F201F4A1E
:1072400080F8401090F937501378214A012D0DDD58
:1072500014465E07A46804D544F0080403E028E05F
:1072600015E024F00804946080F83510B5F1FF3F74
:107270000ADA5B07936802D523F0080301E043F0C4
:107280000803936080F83510F0BCFBF743B890F822
:107290004F1001290DD1B0F8721043F60953491C63
:1072A00089B2A0F87210994203D9A0F8722080F830
:1072B0004F20F0BC70470000700A002048010020F9
:1072C000449900084A990008569900085C990008FA
:1072D000A802002010B5D0E900210369114481FB08
:1072E00003318C0244EA93514260D0E9022382FBCD
:1072F0000332940244EA93521144816010BD0000AD
:1073000030B52049204AB1F86A301088C01A80B2DE
:107310000F2836D31088A1F86A001C4D00204FF0CA
:1073200000432A5C940903D00124B4EB921F24D1BA
:10733000D20622D0164A52F820201268134C12347A
:1073400034F81040224201EB000494F9722008D076
:107350000A2A04DB0A6823FA00F4224308E0521CDC
:1073600009E012F10A0F05DC0A6823FA00F4A243CF
:107370000A6002E0521E84F87220401CC0B211283C
:10738000CFD330BDE4050020280700205894000822
:10739000589500082DE9F00779497A480A89038849
:1073A0009A1A92B2082A74D300880881A1F12C009D
:1073B00042890AB1521E4281734A92F82820802ADB
:1073C00067D302F03F020A70C2890AB1521EC2811D
:1073D000B1F90620902A0CDB8A46FF2A09D08146A3
:1073E000C089002855D1694800230078092805D0B4
:1073F00005E0BDE8F007624800F09EB90823644A42
:1074000092F8EA500DB143F004036248817AC9074B
:1074100001D043F00203D2F808C05FEA0C5101D555
:1074200043F00103176800215B4EFC0302D596F878
:10743000654004B18021C4885FEA446801D541F009
:1074400040015FEA845801D541F020015FEAC47829
:1074500001D041F01001007A400701D541F0080148
:107460004E480078C00701D041F00401A00601D5C4
:1074700041F001010020012D00D1082096F8705044
:1074800085B992F84620022A04D0012A05D03AB1E3
:1074900008E072E040F0030004E040F0020001E088
:1074A00040F001007A0701D440F02000CCF3C00284
:1074B0000025CCF3002C624502D13A0700D4042504
:1074C00096F86F20012A01D145F00105344A0027C2
:1074D000BC4612783E46C2F38102012A04D0022A39
:1074E00004D0032A04D004E0022602E0042600E0CF
:1074F00010262C4A64060ED5214C1C342478240610
:1075000009D51478640606D4274A40F6CC44926D17
:107510006243140C05E0B2F8AE2040F699146243C1
:10752000940B4FF008088AF80A804FF061088AF837
:107530000B808AF80C308AF80D108AF80E008AF851
:107540000F508AF81070270A4B4083F069014140C0
:1075500069408AF8117079408AF8124061405246B9
:107560008AF813C071408AF8146051754FF4C871DD
:10757000A9F80E10FF20AAF80600BDE8F007704732
:10758000E406002028070020E40500201F07002053
:10759000A80200205C0A0020BC0C00204C0900203E
:1075A000CC040020480100201C08002051488169BB
:1075B00041F0FC0181614FF4A060FCF77DF9FBF71D
:1075C00083F9FCF7DDFAF9F7EBFAFCF7D3F8FDF7EE
:1075D000BBF9FFF73DFBFCF713F8FFF7C5FBFBF723
:1075E000E5F8454D45494FF40050A5F81601886768
:1075F000FEF7F0FD00214FF4FA5340F2EE22002096
:10760000401C80B29842FBD3491C89B29142F6D308
:107610003B48002680F87260F9F758F9F9F706FE42
:10762000FCF7DEFAF9F7CCFCFEF7CAFE102235496A
:107630003548F8F7A8FD01F0F7F9344C354FE088EC
:1076400020F04000E0803248017821F020010170F4
:10765000FA20F8814FF49670E887FFF7F5F92E4984
:107660002E48FCF73AFA2E48FCF75CFA2D48416A9E
:1076700088472D48416B8847FEF7DAFF2B48FAF719
:1076800005FA2B494220C8802A49C8603E71E0882B
:10769000E0812089208260896082FAF7FBFCFAF79A
:1076A0005DFCFFF761F801F05FF9FFF7C5FB00F043
:1076B000FBF9FFF725FE01F01BF8FEF7A3F9FAF737
:1076C000B9FAFBF7F3FAFFF71BFAFCF7C5FCFAF778
:1076D00015FFFAF747FF00F07DF8FFF75BFE134850
:1076E000FAF79CF800F06CFAFDF772F9FAF704FA71
:1076F000CDE7000000100240A80200206400002036
:1077000034050020BC0C0020240600205C0A002068
:10771000480100201C070020C8080020980800200D
:107720000C04002038000020E4000020DC090020C8
:107730004807002040040020F0B523490278B0F942
:10774000064000231F4E31F81210FF2C18D0B0F95C
:1077500004701E4DBC4231DA00EBE40704F007046C
:10776000BF7AA7408478FFB23CB190F801C0ACF179
:10777000010C64451FDA3C061DD455F822200DE0AB
:1077800056F82220116012498A79521CD2B28A71AD
:10779000022A02D38370C3808B71F0BD116081789F
:1077A000491CC9B2817042789142F6D38370C18876
:1077B000491CC180F0BD56F82220EFE755F8222081
:1077C0001160F4E7389600086A940008E095000814
:1077D000B8060020F0B561486149B0F86C200B880C
:1077E0009A1A92B29C2A7BD30988A0F86C105D4942
:1077F0005D4F91F82A1001F0070297F84610022A0F
:1078000000D1491E594C80F83E104FF00203E28827
:107810004FF00001550401D5012236E0A489E506A8
:1078200001D5062231E0250701D508222DE05506B5
:1078300003D44F4D2D78AD0601D5042225E0150562
:1078400001D5072221E0150601D50A221DE0950683
:1078500001D50C2219E0150701D50B2215E05507BB
:1078600001D4D50501D510220FE0D50601D505229A
:107870000BE0650703D4A50701D4E40702D080F824
:107880006E3007E0920403D5032280F86E2001E0F9
:1078900080F86E10374A384C92F820E0324A251FA3
:1078A000D2F808C02D4AB2F87060721C92B2BEF1D4
:1078B000000F0DD02CF4000CC7F808C090F86E70C3
:1078C000B7B11E2F1AD090F86F200AB325E007E059
:1078D0004CF40006BE60A0F870200A2A01D2236092
:1078E000F0BD142A01D22B60F0BDA0F87010F0BDDD
:1078F0002B60A0F8701080F86F10F0BD642E04D2D9
:10790000A0F87020322AEED3E9E7A0F87010EAE779
:107910007F1C80F86F70A0F8701090F86F20012A1B
:1079200010D0002AE9D0B0F87060761CB6B2A0F88A
:1079300070601E2ED7D323603C2EDED9521E80F8F5
:107940006F20D2E7B0F87020521C92B2A0F87020DD
:107950002360C82AD1D980F86F10C6E7E40500205B
:1079600028070020BC0C0020A80200205C0A002090
:1079700048010020CC040020141C0140F0B542480E
:10798000B0F84810491C89B2A0F8481002297AD3EF
:107990003E490024A0F848400A783D4B042A57D0BD
:1079A0004FF48041082A0BD0A0F10C02B2F900205C
:1079B0008A4200DA1146B3F980208A4200DA114681
:1079C000344A92698A4200DA11B2418282881D8A61
:1079D000C2EB8502304D12B22D78C5F381062A4DD7
:1079E00042F291767243B5F9765092126A431213BD
:1079F000C26086681546C6EBC60642F3D102F6029F
:107A000002EBA6328260C66C1644C664B0F85070B1
:107A10007F1CBFB2A0F85070B7F5806F04D3B612C8
:107A20000682A0F85040C464891A1C4EC26A724390
:107A300040F255564E4302EB4602466A32444262D9
:107A4000B3F93030B2EB034F06DD1A04426206E0B0
:107A50001349B1F90410B3E7002A00DA4462C162A5
:107A6000104990F83D2091F838108A420BD080F8E8
:107A70003D10B0F84210A0F84410B0F84010A0F843
:107A80004210A0F84050F0BD340500201F07002030
:107A9000A8020020540C0020CC040020C3F5FFFFF6
:107AA000700C00204801002015481649B0F85A20F3
:107AB0000B889A1A92B20F2A20D30988A0F85A107C
:107AC000B0F9001041F6515251438913A0F86C10DF
:107AD0000D494FF480420B78A0F10C01022B06D126
:107AE000B1F90030934202DA1B1D0B8000E00A80DE
:107AF0000021A0F8601020F85C1F42807047000051
:107B000034050020280700201F0700204FF6FF72D1
:107B100002EA800210F4404315480ED0B3F5804FBE
:107B200014D0B3F5004F4FEA122216D0C2F580737D
:107B300030F813305B424B8005E0120A30F8123007
:107B40004B80C2F5807230F812000FE0120AC2F5C5
:107B5000807330F813304B8005E030F81230C2F5F6
:107B600080725B424B8030F81200404208807047C0
:107B700054920008104A518A908AD28A163846399F
:107B8000A2F1110200D54942002A00DA5242114402
:107B9000002800DA40420844084943F6284300B26E
:107BA000B1F936205A43921340F2D733584302EBCF
:107BB000A030C88670470000A802002034050020CD
:107BC000F0B5904990480A8903889A1A92B23E2AE1
:107BD0001ED30088088101F138004FF4FA63428A0D
:107BE0009A4202D2521C428200E04382874A92F8B3
:107BF0002220802A0CD302F03F020A70B1F906203D
:107C0000402A06DBFF2A04D0C2883AB1521EC28045
:107C1000F0BDBDE8F0407B48FFF78EBD428A9A4236
:107C2000F6D307784FF0010E3A074FF0FF055BD50A
:107C3000847A40F2DC52630708D444F00403837270
:107C4000C28081F80BE081F80AE04CE04378072B12
:107C500005D0032B03D0052B01D0062B07D16606D8
:107C600005D444F040038372C280052239E0654A9E
:107C70005FEA437C02F138024FF42076127A0DD588
:107C80005FEAC26C0AD45FEA446C07D442F0100287
:107C900002723A0628D4C680192222E0DF0709D0F2
:107CA000970707D4670605D442F002020272C68025
:107CB000042216E09F0709D5170707D4670605D4E5
:107CC00042F008020272C68003220AE01B070BD5AD
:107CD000530709D4630607D442F004020272C68037
:107CE0000B22CA728A72CD80494AB2F92230B2F9A7
:107CF0001A7003F23D140022A74200DB0276414EC7
:107D0000444C06F13806A479B6895FEAC46C06F1E2
:107D100001064FF4C874B6B213D58681B6F57A7FE2
:107D200005D9017A21F0800101728281F0BD037AC8
:107D30001E06FBD4828143F080020272C4801120AF
:107D400035E09F4216DA037E052B13D28681B6F505
:107D5000487F04D98281027A22F040020272027ABC
:107D60005606E3D45B1C037642F040020272C480E4
:107D700002201CE0284B1C89C4F3C006C4F3002772
:107D800040F2EE24BE4216D11E78360713D4427E4E
:107D9000012ACBD1428BB2F5167F02D2521C42830C
:107DA000F0BD827A42F002028272C4800F20C87253
:107DB0008872CD80F0BD93F80D714FF40046012F0D
:107DC00018D1164F41F6583C7F6C674512DD83F899
:107DD0000CE1134B1E60C38AA34202D25B1CC38218
:107DE000F0BD4FF4FA73C3801C23CB728B72CD802D
:107DF000C282F0BDC2820A4883F80C21001F0660CF
:107E0000F0BD0000C806002028070020E40500207F
:107E1000CC0400205C0A0020A802002048010020B9
:107E2000140801402DE9F05FFE48FF49DFF8FCA38C
:107E3000007E0A1D131D012850465AD030F85A4FB3
:107E40000C8041881180BAF85E001880FDF770FE42
:107E5000F74DF84C49F2CD32B5F91E006083B5F903
:107E6000201043F6CC4C00EB410151430914A1838F
:107E7000B4F92230B4F9206001FB03F200FB0622C2
:107E800042F38F326282B4F9167007FB0CF7BF130E
:107E900040F2333C714302FB0CF200FB131007EB82
:107EA000A232E28240F38F30A082B4F91810E24F80
:107EB000C1EBC10141F3D10101EBE000DF4E2083B2
:107EC000786C3060316930468847DD4930894880B8
:107ED0000846FDF70FFFDFF86CB301264FF00009ED
:107EE0009BF8000008280CD0618F218204287DD0E7
:107EF0001AE030F8604F0C8041881180BAF86400B5
:107F0000A3E7D14890F93710491C02296FD890F89F
:107F1000741019B1B4F85A00208205E0618F2182F3
:107F2000A4F85A1080F87460B4F91410B4F90A0077
:107F3000C64AF9F7B5FAE062BAF91611884204DDCB
:107F4000C248E162027C91408162BA48DFF800E3F6
:107F5000503847F2A30802784EF24611002A79D031
:107F6000012A78D080F800909BF8000004287FD088
:107F7000B64AB4F91210B4F90800303AF9F790FA99
:107F800043F26661A062884200DBA162A3462546F7
:107F9000A06AAE4C443C2060E86A60602046103520
:107FA000FCF734F8A34928883C39FFF7AFFDDFF828
:107FB0008482A8F15008D8F81410C8F87010B5F9E8
:107FC0001010A068B5F9123000FB01F7E2685843C1
:107FD00002FB137444F38F3702FB0100AF8740F3B9
:107FE0008F34EC879B4D6F80AC8001E03DE03AE040
:107FF0002846FEF757FA287F08F11805012878D09F
:10800000604241104DF6B350474369803A142A80CC
:108010004046A8F804408B18C380891AA8F80810B5
:108020008AF80C90B8F904305446002B00DD267312
:10803000B8F90600002802DD217B891C2173B8F9FC
:108040000820002A02DD217B091D2173217B0729DD
:108050007ED202E011E036E00AE0DFE801F0807C49
:10806000947A907E9200608F56E7686A0014E0620E
:10807000B87AE8B37848A06288E7B5F91E20424490
:108080008A420AD8B5F9202042448A4205D8B5F977
:10809000222042448A427FF667AFA0F80290B7F8E8
:1080A000AE204946B2F5C87F01D8467006E0B2F569
:1080B000487F01D8022200E0032242708AF80F10A4
:1080C0008BF8001027E080F80090B5F91EC04A46F2
:1080D000C4448C4509D8B5F920C0C4448C4504D8A3
:1080E000B5F9225045448D42D5D9B7F8AE1001E01C
:1080F0001AE01CE0B1F5C87F01D8467006E0B1F582
:10810000487F01D8022100E00321417042808AF8B3
:108110000F208BF80020BEF8061041F40061AEF885
:108120000610F9F70DFF1FE74FF4AF70A3E74948BA
:108130004DF6B352B0F92030594249106980B0F978
:108140001E00504302142A804046A8F8043062E71B
:1081500005E0667303E0022100E0032161739BF8F0
:1081600000103E4E01293E4F617BDA460DD00729B3
:1081700078D2DFE801F077FEFDFCFBFAF90004217C
:10818000ECE70521EAE70621E8E70729F0D2DFE876
:1081900001F069042F7FA4D8F10001461846FBF7CF
:1081A00083FC2860B5F9020040F6815148438113F1
:1081B0006980B5F9000040F6815250438013288051
:1081C0000A18A2F68152B8F80E305242C3EB62028E
:1081D00012B2A8F80C20002A01DCA8F80C90B8F81C
:1081E0000C20A4F85E201144A4F85C10084479E146
:1081F000404201B2504200B2FBF756FC2860B5F98C
:10820000020040F68151484380136880B5F90010A0
:1082100040F68152514389134218A2F681522980B7
:10822000524220E0DC090020342C0140A80200204A
:108230003405002064000020480100204004002094
:10824000FC0300201F070020700A0020C80800203F
:108250005C0A0020100A0020A2FEFFFF002401405B
:1082600000280140DDE0B8F80E30C3EB620212B224
:10827000A8F80C20002A01DCA8F80C90B8F80C2013
:1082800058E13046F8F7EAFC01231A460721BDE021
:1082900019461046FBF708FC2860B5F9020040F6C5
:1082A0008151484380136880B5F9001040F681522F
:1082B0005143891329804218A2F68152B8F80E3032
:1082C0005242C3EB620212B2A8F80C20002A01DC71
:1082D000A8F80C90B8F80C2059E15942404209B274
:1082E00000B2FBF7E1FB2860B5F9020040F68151CE
:1082F000484381136980B5F9000040F6815250432C
:10830000801328800A18A2F68152B8F80E30524223
:10831000C3EB620212B2A8F80C20002A01DCA8F814
:108320000C90B8F80C20A4F85A201144A4F85C1062
:10833000084462E13046F8F791FC01231A46052112
:1083400064E01146FBF7B0FB2860B5F9020040F687
:108350008151484381136980B5F9000040F681528C
:1083600050438013288006E080E154E125E1F6E0E7
:10837000C6E099E017E00A18A2F68152B8F80E306C
:108380005242C3EB620212B2A8F80C20002A01DCB0
:10839000A8F80C90B8F80C20A4F85C201144A4F8BC
:1083A0005A10084454E1504201B2584200B2FBF75F
:1083B0007BFB2860B5F9020040F6815148438113E8
:1083C0006980B5F9000040F681525043801328803F
:1083D0000A18A2F68152B8F80E305242C3EB62027C
:1083E00012B2A8F80C20002A01DCA8F80C90B8F80A
:1083F0000C20A4F85C201144A4F85E10084455E158
:108400003046F8F72BFC01231A4606213846F8F7C8
:1084100025FC01213046F8F797FB01213846F8F793
:1084200093FBB04EBAF8080055463080BAF80A00FF
:108430007080BAF81000B0803046F9F73BFAB4F813
:108440005A00F1880844A4F86000B4F85C0031894F
:108450000844A4F86200B4F85E0071890844A4F8E6
:108460006400317EA048012978D034F85A1F018079
:1084700061884180A18881809B49028808310A80F7
:1084800042884A80808888809748896A083088476F
:1084900095F83E0000287DD0F8F7E4FD15F83E0F72
:1084A000401E2870BDE8F09F01461846FBF7FCFA15
:1084B0002860B5F9020040F6815148438013688076
:1084C000B5F9001040F68152514389134218A2F6C3
:1084D0008152524252082980A4F85E201044A4F828
:1084E0005C000844A4F85A0000213046F8F72CFB41
:1084F00000213846F8F728FB01231A460621C0E67A
:10850000404201B2504200B2FBF7CEFA2860B5F902
:10851000020040F68151484380136880B5F900108D
:1085200040F68152514389134218A2F681525242B9
:1085300029805208A4F85E201044A4F85A00084488
:10854000A4F85C0000213046F8F7FEFA0021384616
:10855000F8F7FAFA01231A46052192E6B4E0194623
:108560001046FBF7A1FA2860B5F9020040F68151E8
:10857000484380136880B5F9001040F6815251439A
:1085800089134218A2F68152524229805208A4F857
:108590005A2000E09BE01044A4F85E000844A4F8D0
:1085A0005C0000213046F8F7CFFA00213846F8F792
:1085B000CBFA01231A460721BCE65942404209B2D0
:1085C00000B2FBF771FA2860B5F9020040F681515C
:1085D000484380136880B5F9001040F6815251433A
:1085E00089134218A2F68152524252082980A4F8F7
:1085F0005A201044A4F85C000844A4F85E0000214E
:108600003046F8F7A1FA00213846F8F79DFA012321
:108610001A4606218EE61146FBF746FA2860B5F9A0
:10862000020040F68151484380136880B5F900107C
:1086300040F68152514389134218A2F681525242A8
:1086400052082980A4F85C201044A4F85A00084479
:10865000A4F85E0000213046F8F776FA002138468B
:10866000F8F772FA01231A460521C9E6504201B211
:10867000584200B2FBF718FA2860B5F9020040F63C
:108680008151484380136880B5F9001040F681524B
:10869000514389134218A2F681525242520829804E
:1086A000A4F85C201044A4F85E000844A4F85A0022
:1086B00000213046F8F748FA00213846F8F744FA26
:1086C00001231A4607219BE634F8601FCFE60748CE
:1086D0000088A0F5D04168393FF4E4AEBDE8F05F12
:1086E000F9F77CBBDC09002030000020182C014089
:1086F0002DE9F041904C9148B4F85A100288511A73
:1087000089B20F296FD30088A4F85A008C480088DA
:10871000DFF83082C0074FF000054FF0010741D06D
:10872000874AD4E90C1024321388B1EB530F02D2DC
:108730001288511A08444FF4F371884200D2084657
:108740008149B1FBF0F0616CC1F351010844064668
:108750006064F7F762FE00227C4BF7F7CAFD4FF02A
:1087600040427B4BF7F7C5FD0E22F7F731FEF7F7D6
:108770008BFEA4F8A40094F86500401CC0B284F8F5
:108780006500082834D36C4898F84620001F037809
:108790009A4201D0027045806E4A13786E4A23B126
:1087A000458021E06564A56458E0D8F89410A1F5EF
:1087B000FA618E4211DD616D8B1C9E4205DDB0F9C0
:1087C00002100A290DDA491C06E08E4205DAB0F9DA
:1087D0000210002908DD491E4180B0F902000A2874
:1087E00002DB177001E0A2E01570666584F8655041
:1087F0005A484FF4A5420178C1F38101012949D0BB
:1088000002294AD044F687712181A4F8A020B0F94A
:10881000243089B24B439B13A4F89C30B0F90E006E
:1088200000237043B0FBF1F0A16CC0F3D100C1EBA9
:10883000C101C90200EB9130A064F017810341EA45
:108840009641B003F7F76EFCB4F8A210C1EBC1017A
:10885000C902C00800EB9130A4F8A200616CA06EC0
:108860000844A06694F86C20521CD2B284F86C20A4
:10887000082A05D3C008A4F86E0084F86C50A566D9
:108880003748384EC3885A0633D498F80F20022A46
:1088900006D02CE043F20451B6E744F24621B3E798
:1088A000B26840F69916B24221DD94F8382094F867
:1088B0008660B2420CD084F8862094F83D2002F005
:1088C0000106C2F34002964202D1A4F8825004E0AD
:1088D000B4F88220B2F5966F05D2B4F88200401C3D
:1088E000A4F8820005E043F08002C28001E0A4F811
:1088F0008250114894F83F30B0300C2B01D2C5742F
:1089000000E0C774174A0F4C41F2482692F83C2009
:10891000B4F8824041F2504C0C2B0AD3B14208DB30
:10892000012A06D0614502DD002C00D18774BDE824
:10893000F0818574FBE70000480100202807002033
:1089400000040040A80200204564BD0100209C40B6
:10895000133B3340FA030020FB030020CC0400202B
:108960005C0A00203405002070B5284C2848218876
:108970000288511A89B23E2947D3008820802548B1
:10898000808B254D800228606969284688472349E5
:10899000A868FDF78BF822496060CB885A072ED46F
:1089A0000022B0F1F05F0FD9E089B0F5FA7F08D965
:1089B00043F00400C8801B48017821F002010170D7
:1089C0001CE0401CE0811AE0B0F1D25F0CD94FF4FA
:1089D000F031A1EB10308003C910B0FBF1F0206141
:1089E00000280CDA22610AE0B0F1C85F03D94FF425
:1089F0008040206103E023F00400C880E281D4E9D4
:108A00000401884200DB0846A06170BD540C0020C0
:108A100028070020A8020020900600204C9800089B
:108A20005C0A0020DE05002005494FF480404861C3
:108A3000086188610348C18821F48271C180704750
:108A4000540C00205C0A00202DE9F041384C394ECE
:108A5000394F207841F23331C2074FF000050CD076
:108A6000A28962B394F90700002800DA4042C0B23C
:108A7000032829D240F2AE702AE0A570E5732F4A90
:108A8000E571A58192F83830237220F00800A180AA
:108A900040F0020020703D867560B560F560916C15
:108AA000490005D041F68461A18140F0100020709A
:108AB000C0B240F0010020706574BDE8F0816581AE
:108AC00020F01000207015E0042803D240F6510079
:108AD00060810FE0052802D240F69910F8E740F6D1
:108AE000CC42062803D3072801D3082801D262818B
:108AF00000E0618197F89D0098B9B088102301B219
:108B0000B4F90A003622FCF719F87060F168401ACF
:108B1000B1680844B060B6F900104843C013F06073
:108B20003886388E10B10120A070C6E7A570C4E762
:108B3000700C0020A8060020A80200204801002098
:108B40002DE9F041554C2678F0077CD05448217A25
:108B5000544D90F8380081427BD0534A2346DFF8C9
:108B60004CC1575C93F90E2093F90730874203D02C
:108B70001CF80170874213D146F002065B1C267078
:108B80005BB2E3711CF80110814201D15B1CE371FF
:108B900094F90710062901DD0621E171521C1CE041
:108BA000434F17F801C0434F844503D017F801C065
:108BB000844513D126F002065B1E26705BB2E3717A
:108BC000795C814201D15B1EE37194F907306FF04B
:108BD00005018B4200DAE171521EA273207294F9F2
:108BE00007108A1C042A02D941F68462A2812C4A09
:108BF000012912780ADD2B4B56079B6802D543F0FA
:108C0000080301E023F00803AB606070B1F1FF3F9F
:108C100009DA5107A96802D521F0080101E041F005
:108C20000801A9606070F9F775FBA078012810D1E0
:108C300021488068A3280CDA94F90700022803DD94
:108C40000220E07105E01EE06FF00101884200DAC9
:108C5000E171A089002630B1401E0004000CA08103
:108C600001D1E671A673E87B04280CD0B5F9301069
:108C7000512341220020FBF761FF2886002802D102
:108C8000E07B10B1A670BDE8F0810C4806700C487E
:108C90000670207820F001002070F4E7700C0020AE
:108CA00048010020A8020020449900084A990008C1
:108CB000569900085C990008340500203C07002004
:108CC0001F070020743F713D9B3BED396238F4363D
:108CD000A13565343F332A32273133304C2F722E81
:108CE000A32DDF2C242C722B000000361C0700382B
:108CF000AA0A003AAA0A003CCC0C003ECC0C004068
:108D0000380E0042380E0044380E0046380E004837
:108D1000380E004AC711004CC711004EC711005051
:108D2000C7110052C7110054C7110056C71100588F
:108D3000C711005AC711005CC711005EC71100605F
:108D4000C7110062C7110064C7110066C71100682F
:108D5000C711006A00000036220200388E03003A74
:108D6000B005003CD207003EF4090040160C00425A
:108D7000380E00445B100046C71100483313004A08
:108D80009F14004C9F14004E0B1600507717005292
:108D90007717005477170056771700587717005A3F
:108DA0007717005C7717005E77170060771700620F
:108DB0007717006477170066771700687717006ADF
:108DC00000000036FA04003C6606003ED207004070
:108DD0003E090042F4090044AA0A0046600B00481C
:108DE000160C004ACC0C004C820D004E380E005080
:108DF000EE0E0052A40F00545B10005611110058E3
:108E0000C711005A7D12005C3313005EE913006045
:108E10009F140062551500640B160066C1160068A9
:108E20007717006A2D18006CE318006E00000034FC
:108E300000000036000000380000003A0000003C4E
:108E40000000003E0000004000000042000000441E
:108E500000000046000000480000004A0000004CEE
:108E60000000004E000000500000005200000054BE
:108E700000000056000000580000005A0000005C8E
:108E80000000005E0000006000000062000000645E
:108E90000000006600000068441458585870111112
:108EA0005858587041115858487011144858587003
:108EB0001411584858703313005695130054B613C4
:108EC00000525A140050FD14004EA115004C4516D6
:108ED000004A761600486C17004672180044BA190A
:108EE0000042741B0040911D003EB420003C9F22B4
:108EF000003AE1220038532300368B2400348125C8
:108F000000322B2700302028002E5829002CB02AB0
:108F1000002A9B2C0028D22D00267C2F00242631ED
:108F2000002202330020FD34001E5C37001CCC3CC4
:108F3000001A873E0018BE3F001600400014004093
:108F40000012004000100040000E0040000C0040E5
:108F5000000A0040000800400006004000040040F5
:108F6000000200400000002000720020007000207D
:108F7000006E0020006C0020006A002000680020C5
:108F800000660020006400200062002000600020D5
:108F9000005E0020005C0020005A002000580020E5
:108FA00000560020005400200052002000500020F5
:108FB000004E0020004CA320004AA3200048472177
:108FC0000046EB210044EB2100428F2200408F221B
:108FD000003E7A24003C7A24003A66260038512864
:108FE00000343D2A0030702D002CA33000287A3444
:108FF000002451380020CC3C001C004000180040E8
:109000000014004000100040000C00400008004028
:1090100000040040000000000102030405000500F8
:10902000010203040104000305020000F001000036
:1090300036010000F8000000BA0000007C000000CB
:109040007C0000007C000000411414111114441134
:10905000141441110000290052007B00A400CC0030
:10906000F5001E01470170019901C201EA011302D6
:109070003C0265028E02B602DF0208033003590388
:109080008203AA03D303FB0324044C0475049D0448
:10909000C504EE0416053E0567058F05B705DF0517
:1090A00007062F0657067F06A706CE06F6061E07FA
:1090B00046076D079507BC07E4070B0832085908F7
:1090C0008108A808CF08F6081D0944096A09910912
:1090D000B809DE09050A2B0A520A780A9E0AC40A50
:1090E000EA0A100B360B5C0B820BA80BCD0BF30BB3
:1090F000180C3E0C630C880CAD0CD20CF70C1C0D3C
:10910000410D650D8A0DAF0DD30DF70D1C0E400EF0
:10911000640E880EAC0ECF0EF30E170F3A0F5E0FD3
:10912000810FA40FC70FEA0F0D10301053107510E8
:109130009810BA10DD10FF1021114311651187112D
:10914000A911CA11EC110D122E12501271129212A5
:10915000B312D412F4121513361356137613961352
:10916000B713D713F6131614361456147514941433
:10917000B414D314F214111530154E156D158C1549
:10918000AA15C815E7150516231641165F167C1695
:109190009A16B716D516F2160F172C174917661719
:1091A0008317A017BC17D917F51711182E184A18CE
:1091B000661881189D18B918D418F0180B192619BB
:1091C00042195D1978199219AD19C819E219FD19DA
:1091D000171A311A4C1A661A801A991AB31ACD1A2C
:1091E000E61A001B191B331B4C1B651B7E1B971BB0
:1091F000AF1BC81BE11BF91B121C2A1C421C5A1C6A
:10920000721C8A1CA21CBA1CD21CE91C011D181D50
:10921000301D471D5E1D751D8C1DA31DBA1DD01D63
:10922000E71DFD1D141E2A1E401E571E6D1E831EA7
:10923000981EAE1EC41EDA1EEF1E051F1A1F2F1F1A
:10924000451F5A1F6F1F841F991FAE1FC21FD71FB4
:10925000EC1F002000006400C9002D019201F701FD
:109260005B02C00224038903ED035204B6041A050D
:109270007F05E3054706AB060F077307D7073B08D3
:109280009F0802096609C9092D0A900AF30A560BBC
:10929000B90B1C0C7F0CE20C440DA60D090E6B0ED5
:1092A000CD0E2F0F900FF20F5310B4101511761131
:1092B000D71138129812F8125813B81318147714DB
:1092C000D61435159415F3155116B0160E176B17E5
:1092D000C91726188318E0183D199919F519511A5C
:1092E000AD1A081B631BBE1B181C731CCD1C261D4E
:1092F000801DD91D321E8A1EE31E3B1F921FEA1FCE
:1093000041209820EE2044219A21EF2145229922E4
:10931000EE2242239623E9233C248F24E2243425A1
:109320008525D72528267826C82618276827B72711
:1093300006285428A228EF283D298929D629222A3F
:109340006D2AB82A032B4D2B972BE12B2A2C722C3C
:10935000BB2C022D4A2D912DD72D1D2E632EA82E0C
:10936000EC2E302F742FB82FFA2F3D307F30C030C5
:10937000013141318131C13100323F327D32BA3267
:10938000F73234337033AC33E73322345C34953402
:10939000CE3407353F357735AE35E4351A3650369D
:1093A0008536B936ED36203753378637B737E93744
:1093B000193849387938A838D738053932395F39FA
:1093C0008B39B739E2390D3A373A603A893AB23ACD
:1093D000DA3A013B283B4E3B733B983BBD3BE03BBD
:1093E000043C263C483C6A3C8B3CAB3CCB3CEA3CD6
:1093F000093D273D443D613D7D3D993DB43DCE3D18
:10940000E83D013E1A3E323E493E603E763E8C3E8D
:10941000A13EB53EC93EDC3EEF3E013F123F233F39
:10942000333F433F513F603F6E3F7B3F873F933F1A
:109430009E3FA93FB33FBC3FC53FCD3FD53FDC3F3B
:10944000E23FE83FED3FF13FF53FF93FFB3FFD3F96
:10945000FF3FFF3FFF3F0000E7382C35002020EFA3
:109460002037202333202620210000800200040022
:1094700008001000000200040008040000020004BC
:109480000008001000200040008004000000008060
:109490000000004000000020000000100000000854
:1094A0000000000400000002000000010000800035
:1094B0000000400000002000000010000000080034
:1094C0000000040000000200000001000080000015
:1094D00000080140000C0140000C0140000C01405C
:1094E000000C0140000C0140000C0140000C014048
:1094F0000010014000100140001001400010014028
:109500000010014000100140001001400010014017
:109510000014014004080140040C0140040C014007
:10952000040C0140040C0140040C0140040C0140F7
:10953000040C0140041001400410014004100140DB
:1095400004100140041001400410014004100140C7
:10955000041001400414014008080140080C0140B7
:10956000080C0140080C0140080C0140080C0140A7
:10957000080C0140080C014008100140081001408F
:109580000810014008100140081001400810014077
:109590000810014008100140081401400C08014067
:1095A0000C0C01400C0C01400C0C01400C0C014057
:1095B0000C0C01400C0C01400C0C01400C10014043
:1095C0000C1001400C1001400C1001400C10014027
:1095D0000C1001400C1001400C1001400C14014013
:1095E00010080140100C0140100C0140100C01400B
:1095F000100C0140100C0140100C0140100C0140F7
:1096000010100140101001401010014010100140D6
:1096100010100140101001401010014010100140C6
:1096200010140140000000000000000000000000D5
:10963000000000000000000014080140140C01406C
:10964000140C0140140C0140140C0140140C014096
:10965000140C0140140C014014100140141001407E
:109660001410014014100140141001401410014066
:1096700014100140141001401414014000000000B7
:1096800000000000000000000000000000000000DA
:10969000FFFFFF0F0FFFFFFFFFF0FFFFFF0FFFFFB9
:1096A000FFFFF0FF0FFFFFFFFFF0FFFFFF0FFFFFC8
:1096B000FFF0FFFF0FFFFFFFFFF0FFFFFF0FFFFFB8
:1096C000FFFFF0FFFFFF0FFFFFFFFFF0FFFFFF0FA8
:1096D000FFF0FFFF00000040400000000004000019
:1096E00000400000000004004000000000040000F2
:1096F00000400000000400004000000000040000E2
:1097000000400000000004000000400000000004D1
:109710000000004000040000000000808000000005
:109720000008000000800000000008008000000029
:109730000008000000800000000800008000000019
:109740000008000000800000000008000000800009
:109750000000000800000080000800000000002059
:1097600020000000000200000020000000000200B5
:1097700020000000000200000020000000020000A5
:109780002000000000020000002000000000020095
:109790000000200000000002000000200002000085
:1097A0000000006060000000000600000060000093
:1097B00000000600600000000006000000600000DD
:1097C00000060000600000000006000000600000CD
:1097D00000000600000060000000000600000060BD
:1097E00000060000008002000400080010000002D3
:1097F000000400080400000200040008001000201B
:109800000040008004000000FF7FFFFFFDFFFFFF1E
:10981000FBFFFFFFF7FFFFFFEFFFFFFFFFFDFFFF76
:10982000FFFBFFFFFFF7FFFFFBFFFFFFFFFDFFFF5A
:10983000FFFBFFFFFFF7FFFFFFEFFFFFFFDFFFFF74
:10984000FFBFFFFFFF7FFFFFFBFFFFFF0000401F89
:109850007A1903000000001E897603000000C01C76
:109860003BDF03000000801BD15704000000401ABA
:109870009FE00400000000199E7B05000000C01757
:10988000E42C0600000080160DF8060000004015CC
:1098900093DE07000000001408E608000000C01274
:1098A000B1110A000000801101650B00000040109A
:1098B000E6E30C000000000F46940E000000C00D0F
:1098C000467710000000800CB08F12000000400BA3
:1098D000D2DE14000000000A5E6317000000C0081A
:1098E000601A1A000000800726FC1C0000004006D9
:1098F00000002000000000057A1923000000C003CA
:10990000D53926000000800258512900000040018E
:10991000764F2C000000000046252F000000C0FEFE
:109920002AC63100000080FDA1283400000000FBA1
:109930004B1F3800000080F829053B00000000F6AE
:10994000EFFE3C00010203040500020304050001D0
:1099500003040500010205000102030404050001DF
:10996000020355050010AA1A55250030AA3A000036
:10997000AA0A55150020AA2A5535FF3F9C990008D0
:109980000000002054070000E4060008989A000830
:1099900054070020DC09000058670008450204064F
:1099A000082D010203040405480607080913592B72
:1099B0001B086D04211355152A4006190801A71329
:1099C000673D1B088D041A8704012517020604054C
:1099D0000103148020FF8BAA0A02019C15AA0A55D4
:1099E0001500085920AA2A5535FF3F072D03010508
:1099F00004060203127C1573FFFF04FF808001013F
:109A000029025F6402130A13D16A12081201100CB2
:109A10000504060203010103070505280B010203E3
:109A2000040206070303040C3D0706040509191F79
:109A3000191904310506064BAA1A024B381E026991
:109A400010312E40FD3969260211042F405F020CAF
:109A500026405B262ACD55155515123902017F0384
:109A600016D0071AFF01013B0261AA0C1208010877
:109A7000A8147F993F23403313D5720A1608DC914E
:109A8000220312100A17401C12600A16901B014D87
:089A900013E56A020008000062
:020000040800F2
:10FC00004A46545A594D46312D4E3330202020203B
:10FC1000050406020301AA0AAA0AAA0AAA0AAA0A4B
:10FC2000AA0ADE3F00100000FF0131000201664613
:10FC300000400040513800400040004000400101B9
:10FC400000400040FF387B257B257B25FF003333B8
:10FC50000201401F00016626B81E6626FFFFFFFF57
:10FC6000FFFF01010100010001000300000200008C
:04FC70000000AA5591
:04000005080000ED02
:00000001FF
